:10000000B8C300000C943D31D1C30000CFC3000041
:10001000CDC30000CBC30000C9C30000C7C30000AC
:10002000C5C30000C3C300000C94732F0C945B3055
:100030000C94282FBBC30000B9C30000B7C3000055
:10004000B5C30000B3C30000B1C30000AFC30000DC
:10005000ADC300000C944F2FA9C30000A7C300003C
:10006000A5C30000A3C30000A1C300009FC30000FC
:100070009DC300009BC3000099C3000097C300000C
:1000800095C3000093C3000091C300008FC300001C
:100090008DC300008BC3000089C3000087C300002C
:1000A00085C3000083C3000081C30000050109026D
:1000B000A10185020901A1000509190129081500FE
:1000C0002501950875018102050109300931158165
:1000D000257F95027508810609381581257F9501D0
:1000E00075088106050C0A38021581257F95017572
:1000F000088106C0C005010980A101850319012AF4
:10010000B700150126B700950175108100C0050CD8
:100110000901A101850419012AA002150126A002E6
:10012000950175108100C00660FF0961A101096297
:10013000150026FF00952075088102096315002629
:10014000FF00952075089102C005010906A101056F
:100150000719E029E7150025019508750181029529
:1001600001750881010507190029FF150026FF0008
:100170009506750881000508190129051500250156
:10018000950575019102950175039101C00000006C
:10019000000000000000000000000000000000005F
:1001A000000000000000000000000000000000004F
:1001B000007E0F00D4FFFFFFC700000078000000A2
:1001C00000000000002A2B280000000000000000B2
:1001D000000000000000000029000000002C1E3478
:1001E00020212224342627252E362D3738271E1F7E
:1001F000202122232425263333362E37381F0405A9
:10020000060708090A0B0C0D0E0F10111213141516
:10021000161718191A1B1C1D2F3130232D350405F4
:10022000060708090A0B0C0D0E0F101112131415F6
:10023000161718191A1B1C1D2F3130354C09025B7B
:1002400000030100A0FA09040000010301010009F4
:100250002111010001224400070581030800010962
:100260000401000203000000092111010001222203
:100270000007058203200001070503032000010990
:100280000402000103000000092111010001227B8A
:10029000000705840320000112010002000000088D
:1002A000EDFE60300100010203011C0376006900CD
:1002B00061006C003A0066003600340063003200D2
:1002C00062003300630000001803500072006F00EA
:1002D0006A0065006300740020005A0065006E002B
:1002E000000010034C00650067006F006E00750091
:1002F0007400000004030904167C1E001F00200087
:100300002100220000002B0014001A000800150034
:1003100017000000394104001600070009000A0018
:100320000000E1001D001B00060019000500000090
:10033000E000E300E200207821522C004C002A006B
:1003400027002600250024002300000031001300B0
:1003500012000C0018001C000000340033000F00D5
:100360000E000D000B00000028003800370036009A
:100370001000110000004E004B002E002D002152F5
:100380002C0028003A003B003C003D003E003F00AE
:1003900000000100257827782678007C2F000000D7
:1003A0000100247828782378010001000000E10092
:1003B000010001000100010001000000E000E30075
:1003C000E2002178010001000100450044004300E3
:1003D00042004100400000004A0049004E00520027
:1003E0004B00300000004D004C004F005100500009
:1003F00001000000AB00AC00AE0001000100137072
:100400000000AA00A900A8000100010001000100ED
:100410002223252628292A2C2D2F30323335363811
:100420003A3B3D3E4042434547494A4C4E5051536A
:100430005557595A5C5E6062646668696B6D6F718E
:10044000737577797B7D7F81838587898A8C8E9090
:10045000929496989A9C9E9FA1A3A5A7A8AAACAE99
:10046000AFB1B3B4B6B8B9BBBCBEBFC1C2C3C5C6D9
:10047000C7C9CACBCCCDCED0D1D2D2D3D4D5D6D782
:10048000D7D8D9D9DADADBDBDBDCDCDCDCDCDDDDC0
:10049000DDDDDCDCDCDCDCDBDBDBDADAD9D9D8D7B0
:1004A000D7D6D5D4D3D2D2D1D0CECDCCCBCAC9C752
:1004B000C6C5C3C2C1BFBEBCBBB9B8B6B4B3B1AF89
:1004C000AEACAAA8A7A5A3A19F9E9C9A9896949229
:1004D000908E8C8A89878583817F7D7B7977757300
:1004E000716F6D6B6968666462605E5C5A595755DE
:1004F0005351504E4C4A4947454342403E3D3B3A9A
:100500003836353332302F2D2C2A29282625232220
:10051000FFAA7F5540000101010101010101010213
:1005200002020202020202020303030303030303A3
:10053000040404040404040505050505060606066E
:1005400006070707070708080808090909090A0A2A
:100550000A0B0B0B0C0C0C0D0D0D0E0E0E0F0F0FCE
:100560001010111111121213131414151516161759
:1005700017181819191A1A1B1B1C1D1D1E1E1F20C7
:1005800020212222232424252626272829292A2B14
:100590002C2D2D2E2F303132323334353637383939
:1005A0003A3B3C3D3E3F4041424344454647484933
:1005B0004A4C4D4E4F50515354555658595A5B5D05
:1005C0005E5F616264656668696B6C6D6F707273A3
:1005D0007577787A7B7D7E8082838587888A8C8E0A
:1005E0008F91939596989A9C9EA0A2A3A5A7A9AB3C
:1005F000ADAFB1B3B5B7BABCBEC0C2C4C6C9CBCD2E
:10060000CFD1D4D6D8DBDDDFE2E4E7E9EBEEF0F3DF
:10061000F5F8FAFDFF1E0F0500047F3F1F6432143A
:10062000643214783C1E1E140A05FD377A585A00AD
:100630000004E6D6B4460200210116000000742F23
:10064000E5A3E0024200D65D003D888986D3DC0A3E
:10065000E842C324925842597FBD199EB8FF9AB10F
:100660005C1A1E330845639C1174376FBFEF729795
:1006700018248DBC060AF75D420146E1C168CA47ED
:100680001B77C4B3A03FB66248BF858DB35356985D
:10069000F898A16CDBDA8D54259A04414E88175ED8
:1006A0002513733EAE8E3737C92C01CD182DCB885C
:1006B000DC47535E4DC41B957EE40CCF533F813F16
:1006C0008CF789FFAB5DEEAB109CB1F9928B2438AF
:1006D0001768FADB6981DDA858F86B7BF4EA2B6CAC
:1006E000136FC45131AB4C96238158874425DBC529
:1006F00086DC3E049A2CC2881529274A6324FD55BE
:10070000D3CA16D9D40E1125AB2482104C2C2D46F9
:10071000A8A6DAC4FC43FFFB1B3E0982B04B640071
:1007200000002ACE090DCBF926C30001F201C30453
:1007300000004BAC9EC5B1C467FB02000000000482
:10074000595A504F52514A4D4B4E2A4C2F30B6B742
:10075000ABACBBBCA9AABDBECFD0CDCEDBDCD9DA59
:100760000D0E0B0F1A0508050905071811130408CB
:10077000120C11241FBECFEFDAE0DEBFCDBF24E0A4
:10078000AEEFB1E001C01D92AE30B207E1F711E06B
:10079000A0E0B1E0ECE0FAE602C005900D92AE3FB9
:1007A000B107D9F70E94F7270C94603429CC9C013B
:1007B000FB019A9581159F4120F5832F8170B32FFE
:1007C000B270AA27732F74706627532F587044276E
:1007D00034FF0DC08295807FAB2B09F08062672BC0
:1007E00009F08064452B09F0806809950895AB2BCA
:1007F00009F08260672B09F08460452BB1F38860B3
:10080000F4CF80E0F2CF0C94BC320895982F9295EB
:100810009F7024E0911102C020E0982F892F8695C7
:100820008695811511F02E5F982F892F8695820F5E
:1008300008958093B10308958093B203089521E051
:1008400030E001C0220F8A95EAF78091B203822B33
:10085000F3CF21E030E0A90102C0440F551F8A9573
:10086000E2F7CA0180959091B2038923E5CF292F41
:100870009A3090F5873080F590E037E0239F800D27
:10088000911D1124282F277041E001C0440F2A95A3
:10089000EAF723E0969587952A95E1F7FC01EE0F9C
:1008A000FF1FE80FF91FEB5EFC4F20E030E070E027
:1008B0005191DF01CB01022E02C0969587950A94D3
:1008C000E2F7817081958527842385278E932F5F9A
:1008D0003F4F2330310561F70895292F9A3078F57D
:1008E000873068F590E037E0239F800D911D11243B
:1008F000682F677023E0969587952A95E1F7FC01AC
:10090000EE0FFF1FE80FF91FEB5EFC4F40E050E0D9
:1009100080E0219130E0062E02C0369527950A949A
:10092000E2F721703327042E01C0220F0A94EAF760
:10093000822B4F5F5F4F4330510559F7089580E098
:1009400008959091B20321E030E0F90101C0EE0F6B
:100950008A95EAF7D90102C0AA0FBB1F6A95E2F790
:10096000EA2B01C0220F4A95EAF7892F8E23E8135C
:1009700003C0892F822B60CF2095822F8923FBCF44
:100980008091BA039091B903981301C008958F5FC5
:100990008770FACF9091B403809589238093B40334
:1009A000282F2770211110C0891771F090910D0424
:1009B00092FF0AC08695869586954BDF1092B40308
:1009C0001092B6031092B5030895982F90958091D8
:1009D000AF0389238093AF0308958091AE038115FF
:1009E00031F01092AE031092B8031092B70308953D
:1009F000803E9105D9F1C8F48133910509F482C094
:100A000048F48932910509F472C08A32910509F4DB
:100A100080C0089589339105E9F082389105D1F0BD
:100A20008533910509F45EC00895843E9105D9F19E
:100A300048F4823E910539F1833E910549F181EEFA
:100A400090E00895863E9105C9F1873E910509F42D
:100A50003EC0089520910C042370211164C02091A0
:100A60000D0423FF14C089E290E0089520910C0446
:100A700020FD45C030910D0430FF09C024FD24C085
:100A800083EE90E0089520910C0422FDF7CF0895A5
:100A900020910C0422FD44C030910D0430FD43C070
:100AA00024FFF5CF11C020910D0421FFF0CF8091DC
:100AB0000C0484FD09C087EE90E0089520910C0499
:100AC00023FFE5CF24FFF7CF80E090E00895209149
:100AD0000C0423FD2BC030910D0431FFE1CF84EED7
:100AE00090E0089520910C0425FFD1CFBCCF209138
:100AF0000C0425FD1EC020910D0423FFC8CF89E3FF
:100B000090E0089520910C0426FFC1CF8AE290E086
:100B1000089520910C0426FFBACF81E390E0089558
:100B200082EE90E0089580EE90E0089586EE90E0E9
:100B3000089585E390E0089590910C0492FF10C011
:100B400041E0282F2471243009F040E031E0282FC3
:100B50002871283009F030E0431711F02CE082278B
:100B600093FF10C041E0282F2471243109F040E0A8
:100B700031E0282F2871283109F030E0431711F0B7
:100B80002CE0822730910D0430FF10C051E0282F57
:100B90002171213009F050E041E0282F28712830E0
:100BA00009F040E0541711F029E0822731FF10C00E
:100BB00041E0282F2171213109F040E031E0282F58
:100BC0002871283109F030E0431711F029E082271D
:100BD00094FD877E08951F93CF93DF9309DFEC0187
:100BE000811522E5920708F052C0811540E594076F
:100BF00008F0CDC0803E910520F58D3C910508F0B0
:100C0000A1C0883A910570F4853A910508F097C023
:100C100081309105B9F10497813A910598F1C0E0CE
:100C2000D0E030C0885A91094B97C8F7C85AD0E035
:100C3000CC0FDD1FCE56DE4F0990D881C02DD46475
:100C400021C0811550E49507B0F4C11580E2D807A2
:100C500008F0B3C0C83ED105A8F0CE019A95811521
:100C60009F41E8F68D2F68DF182FCE019927C0DE4F
:100C7000EC01D12B07C09927BBDECC27DF70C82B36
:100C8000D92BD06ACE01DF91CF911F910895803882
:100C900042E59407C8F5803652E5950708F05BC039
:100CA000C03482E5D807D0F4C03292E5D90708F005
:100CB0004BC08C2F8695869520E2829FC00111241F
:100CC000C37021E030E0A90102C0440F551FCA954E
:100CD000E2F7EA01C82BD92BDD68D4CF8C2F86959B
:100CE0008695877050E2859FC0011124C37021E072
:100CF00030E0A90102C0440F551FCA95E2F7EA018E
:100D0000C82BD92BDC68BECF803C52E5950758F440
:100D10008F71C03AD245A0F590E0982F8827EC015A
:100D2000C46FD06AAFCF805C9245809708F077CFD0
:100D3000DC2FCC27CC27DF71C06FD06AA3CFA4975C
:100D4000D064A0CFD0659ECFCF71D0E0DC2FCC2770
:100D5000C16FD06A97CF86958695877020E2829F73
:100D6000C0011124C37021E030E0A90102C0440F8A
:100D7000551FCA95E2F7EA01C82BD92BDA6882CF52
:100D8000DBDEC82FD0E0DC2FCC27D0627BCF8F7189
:100D9000D3DE93E0CC0FDD1F9A95E1F7CC27DF700F
:100DA000282F30E084FF05C050E1859F9001112479
:100DB0003327C22BD32BD06965CF8D2F8F71BCDE2B
:100DC000182FCE01992714DEEC01D12BDECF80E065
:100DD0000895F894E82FE295EF70F0E041A18F704C
:100DE00021E030E0B90102C0660F771F8A95E2F773
:100DF000CB01962F9095942391A392A1892B82A346
:100E0000789408950895CF92DF92EF92FF921F9306
:100E1000CF93DF93172FE82FF0E0EB5EFA4F7111BD
:100E20000CC0E4918E2F7E2F6E2FDF91CF911F91FA
:100E3000FF90EF90DF90CF900895E62EF12CC72E13
:100E4000D12CF491EF2F86E0689F90011124CFEF11
:100E5000D0E0C901BE010E948F32AB01EE0CFF1C35
:100E600065E5649FC001659F900D1124E81AF90A99
:100E70006E2D660F6E0D7E01EC18FD08FE9DD001F3
:100E8000FF9DB00D11248B2F169F70011124EF2CA4
:100E9000FF246E01CE18DF087601FE9D6001FF9DE4
:100EA000D00C11247E01E61AF108B701169F7001DB
:100EB000179FF00C1124EF2CFF24CE19DF09FC9FA3
:100EC0007001FD9FF00C11247F2D43305105C1F0BE
:100ED0002C3F334058F441305105B1F042305105B8
:100EE00009F0A2CFEB2F8F2D7F2F9ECF44305105DD
:100EF00071F04630510509F497CF7B2F8D2D94CF9B
:100F00007D2DEB2F8F2F90CF7F2FED2D8DCFEF2DC0
:100F10007B2FF8CFCF93982F762F842FC22F692F56
:100F200072DF472F282F8C2F90E03CD2CF9108956D
:100F30008091A503843028F4837084608093A50396
:100F400008958C3AE8F38370886AF8CFCF93DF93E3
:100F50008091A50380FD0BC0C0E0D0E020E040E020
:100F600060E0CE011FD22196C031D105B9F779D604
:100F7000DF91CF910895FF920F931F93CF93DF934B
:100F8000182F062FF42E8091A50380FF0CC0C0E01F
:100F9000D0E02F2D402F612FCE0104D22196C031F9
:100FA000D105B9F7D3DFCDB7DEB7E5E00C947532E4
:100FB000CF93DF93EC012091A8039C81892F81704E
:100FC00090FD822F692F627091FD622F492F44702E
:100FD00092FD422FD0DF8C8190E001968770992797
:100FE0008C83DF91CF910895982F762F842F2091B5
:100FF000A50320FF07C0692F06DF962F672F482F14
:10100000892FB9CF0895CF93DF93EC01E5EAF3E0A0
:10101000438162818C81E8DF8C818F5F8C83DF91DB
:10102000CF910895CF93DF93EC01EC81F0E0E05F86
:10103000FB4F4491E5EAF3E062818181D5DF8C8149
:101040008F5F8C83DF91CF910895FF920F931F9351
:10105000CF93DF93EC01F12C00E010E08C8198013C
:101060004091A8036091A7038F0D54DF0F5F1F4FBE
:101070008FE0F80E0031110589F768DF8C819A81C5
:1010800090FF07C08F5F8C83CDB7DEB7E5E00C948F
:1010900075328150F8CFEF92FF920F931F93CF9349
:1010A000DF93FC018281FF24F39480FF02C0FF24C0
:1010B000FA94C0E0D0E020E040E060E0CE0172D1E0
:1010C00004E010E0E12C8091B1028E0D813174F1C9
:1010D0008F70082E001C00088C170D0679F44091C3
:1010E000A8030403A00111245595479555954795EC
:1010F0009E016091A7038091A6030CDFEF0C0150C5
:10110000104009F72196C031D105A9F61FDF809163
:10111000B102F1E0FF120EC0811579F08150809389
:10112000B102CDB7DEB7E6E00C94743287FFD1CFC1
:10113000805FCFCF8F5F8F70F2CF8FE0F0CFCF93F4
:10114000DF93C0E0D0E020E040E060E0CE012AD1B3
:101150002196C031D105B9F7C0E0D0E08091B0024E
:10116000082E001C0008C817D0055CF1809106010C
:10117000082E001C00088C170D061CF19E014091E2
:10118000A8036091A7038091A603C4DE2196C03115
:10119000D10521F7DBDE809105019091B002980F17
:1011A0009093B00220910601280F20930601121699
:1011B00014F49F301CF0819580930501DF91CF914D
:1011C000089520E040E060E0CE01ECD0DFCFA6E063
:1011D000B0E0EDEEF8E00C9456328D839E83AD8145
:1011E000BE811496FC912F2F30E0D9010E9451341A
:1011F0009B01AC010E941F346B017C0180E290E0F6
:101200009C012F1B3109F901A5E5B0E0A70196016A
:101210000E941F3469837A838B839C839F01DF0143
:101220000E94D3329B010E94D9329B01AC012C0D4C
:101230003D1D4E1D5F1D69817A818B819C810E94BD
:101240002F34022F30E00A32A0F5A901440F551FB8
:10125000420F531F55954795142F1095E12CF12CF3
:1012600085E5D82ED01A8D2DE1FC802F9701412FD6
:101270006091A7034FDE3FEFE31AF30A80E1E8161F
:10128000F10489F763DEAD81BE8114969C9181E003
:10129000911519F0903219F48FEF80930401809129
:1012A0000401890FED81FE8184832696E8E00C9489
:1012B000723285E590E0821B930BAC01440F551F01
:1012C000480F591F57FFC6CF4F5F5F4FC3CF0F93D4
:1012D0001F93CF93DF93EC0120E030E06091A703F0
:1012E0008091A6039C8189010F5F1F4F2830310533
:1012F0003CF4911541F04091A8030CDE9801EECF2B
:101300004091A803911140E005DE980100311105DC
:1013100029F71CDE8C8190E00196817099278C83DF
:10132000DF91CF911F910F910895FB01811520E26C
:10133000920728F4811541E0940738F408959C0140
:1013400030522115304348F00895392F94FF02C0E0
:101350003295307F2081232B208399270895462BB7
:1013600022FF0FC0982F92959F708F70892B962F18
:1013700092959F706F70692B942F92959F704F700C
:10138000492B982F9623961309C050E0409550950D
:1013900090E04823592381E0452B09F080E008952F
:1013A000519A0895FC01EE0FFF1FE80FF91FE05D51
:1013B000FD4F61834083228308950F931F93CF9342
:1013C00001E010E0082E01C0000F0A94EAF7C09176
:1013D000AD039C2F9023911115C09091B403969565
:1013E00096959695891306C01092B4031092B60391
:1013F0001092B50324DAC027C093AD03CF911F919B
:101400000F91089526DAF7CF282F35EB2303C0017B
:10141000112497FF04C080589109892F089580589E
:101420009F4FFBCF8091360380FF0DC060913E013E
:1014300070E0660F771F60387105B0F561157105B2
:10144000A9F1862F089581FF07C060913E0184E0D5
:10145000689FB0011124EFCF82FF04C060913E016C
:1014600088E0F6CF909135039115D9F020913D0198
:1014700080913E01682F70E0921730F043E0660FD4
:10148000771F4A95E1F7D7CF899FC001112433E038
:10149000880F991F3A95E1F7622F70E00E94A332FE
:1014A000CACF68E070E0CDCF8FE7089581E008955E
:1014B0008091360380FF0CC060913C0170E075950F
:1014C0006795759567956115710549F1862F0895A2
:1014D00081FF06C060913C0170E075956795F3CF80
:1014E00060913C0182FD0BC0909134039115A1F0F5
:1014F00060913B0180913C01961738F0682F70E0B5
:101500006038710500F38FE70895899FC0011124A9
:1015100070E00E94A332F4CF61E070E0D7CF81E0A9
:1015200008959091920389029001112437FF03C01E
:101530008093920308952F3731051CF4980F9093F0
:10154000920308959C0180E090E0F901E80FF91FF3
:10155000E491E41307C091E08927F901E80FF11D38
:10156000849108950196861780F380E00895809114
:101570000303811569F0E0910B03F0910C033097A0
:1015800039F00190F081E02D309711F00995089520
:1015900080E00895A3E0B0E0E0EDFAE00C945C3266
:1015A0009C0180912E0290912F0282179307B1F037
:1015B00030932F0220932E02E0910B03F0910C0345
:1015C000309761F00084F185E02D309739F083E0A9
:1015D00089833B832A83CE01019609952396E2E015
:1015E0000C947832A3E0B0E0E8EFFAE00C945C32BF
:1015F0009C0180912C0290912D0282179307B1F0EB
:1016000030932D0220932C02E0910B03F0910C03F8
:10161000309761F00084F185E02D309739F084E057
:1016200089833B832A83CE01019609952396E2E0C4
:101630000C947832A2E0B2E0EFEF90E02D918217A7
:1016400051F0EF3F19F4211101C0E92F9F5F96304F
:10165000A9F7EF3F09F408950E2E000CFF0BE050A0
:10166000FE4F82830895E2E0F2E09191891302C077
:10167000DF011E9292E0E830F907B9F708958091F2
:10168000130108952FB7F8948091280290912902B0
:10169000A0912A02B0912B022FBF0895962F20917E
:1016A0000D0422FF0EC0682F660F660F660F692BB0
:1016B0006093B403C4D8E6DF9093B6038093B50378
:1016C0000895BDC89091AE03292F2823211559F004
:1016D000809589238093AE03811531F0D3DF809309
:1016E000B7039093B803089580E090E0F8CFCADF85
:1016F0002091390330913A03232B211521F0809357
:10170000D4029093D50220913B0330913C03232BCC
:10171000211521F08093D2029093D302E0910B0324
:10172000F0910C03309759F00680F781E02D309747
:1017300031F082E08093370387E393E009950895C1
:10174000611509F441C0E3E3E80FE33148F4F0E048
:10175000EE59FB4C0C94B63265DE819580933A03CA
:10176000C6CF60DEFBCF5EDE819580933903F8CF74
:1017700059DEFBCF9DDE80933B03F2CF99DE81954E
:10178000FACF96DE819580933C03EACF91DEFBCFC2
:10179000815D990B21E030E001C0220F8A95EAF7C4
:1017A00080913803822B80933803DACF80913603FF
:1017B000816080933603D4CF809136038260F9CF65
:1017C000809136038460F5CF409139038D3C59F404
:1017D00080913A0387FF0DC010923A03411559F4E6
:1017E0001092350308C08E3C81F480913A0318169C
:1017F0009CF3411581F080913B0390913C03892B30
:101800008111AECF10923403ABCF8F3C41F447FF30
:10181000F0CF1092390380913A038115E0CF803DDB
:1018200019F41416B4F3E5CF90913B03893D29F4E4
:101830001916FCF610923B03DCCF8A3D19F497FF92
:10184000D8CFF8CF90913C038B3D29F497FFD1CFAF
:1018500010923C03CECF8C3D19F41916CCF3C9CFAE
:101860009FE2980F983090F4815D990B21E030E071
:10187000B90102C0660F771F8A95E2F7CB01809508
:1018800090913803892380933803B3CF8D3D31F491
:10189000809136038E7F80933603ABCF8E3D21F44B
:1018A000809136038D7FF7CF8F3D09F0A2CF8091D5
:1018B00036038B7FF0CF2FB7F89460912802709198
:1018C000290280912A0290912B022FBF08950F9335
:1018D0001F9380910303811521F0EDDF1F910F917C
:1018E0000895E9DF0091FF021091000320910103A8
:1018F00030910203600F711F821F931FEFCF809101
:101900000303811509F0BECEE2DFCB01089587E71E
:1019100097E7909301088093000888E19AE00FB65A
:10192000F894A895809360000FBE90936000FFCF5D
:101930000895FC019B0180911E0290911F02861761
:10194000970740F0672B29F48091E8008E77809309
:10195000E800C90140E0009741F4411106C08091C0
:10196000E80082FF2FC080E008952091E702211552
:10197000A9F12530A9F12091E80023FD2DC0209187
:10198000E80022FDECCF2091E80020FFE4CF309169
:10199000F3002091F200009719F02830310558F03B
:1019A00041E02830310509F040E02091E8002E7731
:1019B0002093E800D0CF41914093F10001972F5F31
:1019C0003F4FE9CF8091E702811541F0853041F02A
:1019D0008091E80083FFC3CF81E0089582E00895FD
:1019E00083E008958091180287FF13C08091E8007A
:1019F00082FF06C08091E8008B778093E80008950D
:101A00008091E7028111F2CF08958091E70281155C
:101A1000D9F38091E80080FFF8CF8091E8008E77BD
:101A2000ECCF2091E4003091E50095E6A9012091EA
:101A3000EC00822F817020FF06C08091E80080FFBB
:101A400006C080E008952091E80022FD1AC0809130
:101A5000E702811589F0853089F08091EB0085FDE2
:101A60000FC02091E4003091E50042175307F9F2CE
:101A70009A95E1F684E0089582E0089583E0089560
:101A800081E00895E8EDF0E080818E7F8083109200
:101A9000E2001092DA001092E100A0EEB0E08C912A
:101AA00081608C9380818F77808319BCA7EDB0E033
:101AB0008C918E7F8C9380818F7E80831092170211
:101AC0000895E0910B03F0910C03309739F00284F4
:101AD000F385E02D309711F060E209950895FC013F
:101AE000AC014B5F5F4F8FEF61E39191892728E055
:101AF00030E0982F990F87FF09C0892F8627215042
:101B00003040B9F7E417F50781F70895892FF7CF2B
:101B1000982F9093E900891771F07091EC00209153
:101B2000ED005091F00021FD09C09F5F973089F7CB
:101B30008093E9000895762F242F50E03091EB0038
:101B40003E7F3093EB003091ED003D7F3093ED0010
:101B50003091EB0031603093EB007093EC002093F8
:101B6000ED005093F0002091EE0027FDDECF0895A8
:101B7000A0E0B0E0EEEBFDE00C945632C8EDD0E012
:101B800088818F7E8883E7EDF0E0808181608083AB
:101B900084E082BF81E08093170288818E7F8883F2
:101BA00002EE10E0F80110821092DA0081EEC82EE9
:101BB000D12CF601108288818F7788838881806894
:101BC000888388818F7D888319BC1092E7021092E8
:101BD00016021092C0021092150290EEE92EF12C1E
:101BE000F70180818B7F808388818160888342E0D8
:101BF00060E080E08DDFF60180818E7F8083F801D8
:101C0000808181608083808188608083F70180810A
:101C10008E7F8083888180618883CDB7DEB7E8E0DE
:101C20000C947232E091BA039091B90329E0E91360
:101C300002C080E00895AE2FB0E02E9FF001112485
:101C4000E554FC4F3181361306C03081381303C090
:101C50003581341304C0FD013196E770E8CF81E08F
:101C600008953BB13D7F2BB122604FB7F89480E3DC
:101C700092E0FC010196508168E02BB9000000C0A1
:101C800057FF3BB9550F000000C000C000C03BB972
:101C900000C06A9591F752E08036950751F74FBF23
:101CA0008FE594E00197F1F700C0000008950F93CD
:101CB0001F93CF93DF938B01EA019091E702943059
:101CC00051F58093E9008FEF9091E80095FD06C0F3
:101CD00095ED9A95F1F700008A95B1F78091E800AB
:101CE00085FF19C09EDE811111C08091E80085FD3D
:101CF00006C08091E8008E778093E800F3CFF8016A
:101D000081918F018093F100219779F78091E8000C
:101D10008E778093E800DF91CF911F910F91089506
:101D2000792F603229F440E250E0682F82E0BFCF83
:101D30000895CF93DF93D82FC92F48E050E0682F44
:101D4000792F81E0B4DF88E0ED2FFC2FA0E2B2E034
:101D500001900D928A95E1F7DF91CF910895BC0132
:101D600046E050E084E0A3CFBC0143E050E084E0D3
:101D70009ECFA0E0B0E0EFEBFEE00C945432F82EE2
:101D8000E92EB62EA72E8A01809112029AE0C92E62
:101D9000D12C8A3018F0CC24C394D12CC1E0D0E0EF
:101DA0006B2D7A2D8F2D9E2DF8010995811116C06E
:101DB0002196CC16DD0694F0CC9FC001CD9F900DEE
:101DC000900D112420E030E045E34A95F1F7000042
:101DD0002F5F3F4F28173907B9F7E2CFCDB7DEB7EE
:101DE000EAE00C94703290910D0492FB222720F9C6
:101DF000281779F080FB92F990930D0460910C0400
:101E000070910D0484E090E00E94E83382E00C942D
:101E1000CA0408951F93CF93DF93962F122F632F39
:101E20008330D8F49A30C8F44730B8F4C42FD0E0E7
:101E3000CC0FDD1F2EE0929FC00DD11D11249CE818
:101E4000899FC00DD11D1124CE0189960E94CE33E9
:101E5000612FCE018A960E94CE33DF91CF911F91E0
:101E60000895CF93DF93C091AF038091B303C82B44
:101E70008091AE038115F1F005DC2091B70330911C
:101E8000B803821B930B8838934110F00E94ED0435
:101E9000D091AE0320E082E092E0FC013081019617
:101EA00031112F5F32E088309307B9F721110E947A
:101EB000ED04CD2BC093000248E050E06DE073E0EC
:101EC00080E092E00E948033892BB9F088E0E0E066
:101ED000F2E0ADE0B3E001900D928A95E1F7E09178
:101EE0000B03F0910C03309741F00280F381E02D59
:101EF000309719F080E092E00995DF91CF91089535
:101F0000CF931092AF03C6E0E2E0F2E0DF018C2F46
:101F10001D928A95E9F780E090E03CDB80E090E05C
:101F200061DB1092B3039DDFE7E3F3E0DF011D9275
:101F3000CA95E9F7109235031092340310923603D4
:101F4000D6DBCF910895DCDF2FEF84E39CE02150B6
:101F500080409040E1F700C0000088E19AE00FB6B1
:101F6000F894A895809360000FBE90936000FFCF17
:101F7000AAE2B0E0EEEBFFE00C945B3288E192E085
:101F8000FC0101962091F100208322E0803292072B
:101F9000B9F780911902893009F457C0C8F482302A
:101FA00009F4B2C0833009F482C0813081F180919C
:101FB000E80083FFE6C080911802909119029A30E0
:101FC00008F0DFC0E92FF0E0EB58FB4C0C94B63280
:101FD0008A3009F489C08B3051F780911802813220
:101FE00031F780911C0290911D02892B01F780919D
:101FF000E800877F8093E800F5DC81E090911A0289
:10200000911101C080E0809314017ADFD0CF8091DC
:102010001802813A61F68091E800877F8093E8009A
:1020200080911C0290911D02892B59F060E080E0A4
:1020300090E070E07EDC8091E8008B778093E80090
:10204000B6CF68E080E292E0F4CF8091180281324E
:1020500009F0ADCF80911C0290911D028D7F892BDC
:1020600009F0A5CF8091E800877F8093E8008091F8
:10207000E80082FF17C09091F3008091F200029770
:1020800031F48091F100813011F0863021F480919B
:10209000F100809313018091E8008B778093E80032
:1020A000A1DC85CF8091E7028111E1CF80CF8091C3
:1020B0001802813A09F07BCF80911C0290911D0299
:1020C000892B09F074CF8091E800877F8093E80026
:1020D0008091E80080FFFCCF809114018093F10093
:1020E0008091E8008E77DACF80911802813209F072
:1020F0005ECF8091E800877F8093E80073DC809159
:102100001B028093120153CF80911802813A09F08B
:102110004ECF8091E800877F8093E8008091E800AF
:1021200080FFFCCF80911201D9CF803889F08238AE
:1021300041F580911C028F70873018F58093E9007B
:102140008091EB0085FB882780F91092E90006C09A
:102150008091C002880F90911502892B9091E80020
:10216000977F9093E8008093F1001092F1008091A6
:10217000E8008E7723C0811116C080911A02813049
:1021800009F18091E80083FF0AC08091E800877F11
:102190008093E8008091EB0080628093EB00AA9628
:1021A000E3E00C947732823061F780911A02811556
:1021B00081F01092E9008091E800877F8093E80029
:1021C00011DCDFCF81E0933009F080E08093C00222
:1021D000F0CF80911C028F702FEF280F263088F6E9
:1021E0008093E9002091EB0020FFE3CF933031F49E
:1021F0008091EB0080628093EB00DBCF9091EB004D
:1022000090619093EB0021E030E0A90102C0440FFF
:10221000551F8A95E2F74093EA001092EA008091F8
:10222000EB008860E8CF8111ACCF10911A021F77C4
:102230008091E3008078812B8093E3008091E80017
:10224000877F8093E800CEDB8091E80080FFFCCFA1
:102250008091E30080688093E30083E0111101C066
:1022600082E08093E7028DCF8058823008F089CFDA
:1022700080911A0290911B028C3D53E0950791F5D5
:1022800083E08A838AE289834FB7F894DE0113964C
:1022900020E03EE051E2E32FF0E0509357008491BC
:1022A00020FF03C082958F703F5F8F708A30C0F02F
:1022B000895C90E08D939D932F5F243161F74FBF30
:1022C0008091E800877F8093E8006AE270E0CE01A9
:1022D00001962FDB8091E8008B778093E80051CF47
:1022E000805DE7CF292F33272330310509F44EC015
:1022F00078F52130310509F488C08BE590E0EDE3F5
:10230000F2E02230310509F03CCF2091E800277F30
:102310002093E80020911E0230911F02821793073C
:1023200008F49C0140E02115310509F073C041110A
:1023300071C08091E80082FDCDCF8091E7028115C8
:1023400049F2853039F28091E80083FFF2CFC2CFA5
:1023500080911C0290911D022132310509F446C082
:102360002232310509F00DCF8330910508F009CFF5
:10237000FC01EE0FFF1FE35BFE4F0190F081E02DAB
:10238000865B9E4FDC018C9190E010C09C0133274E
:10239000823021F12330310568F4232BB9F4E4EFC6
:1023A000F2E0E4918E2F90E0E4EFF2E0009709F480
:1023B000E8CEABCF2330310509F0E3CEEAEAF2E014
:1023C000E4918E2F90E0EAEAF2E0F0CFE2EEF2E064
:1023D000E4918E2F90E0E2EEF2E0E8CFE8ECF2E05C
:1023E000E4918E2F90E0E8ECF2E0E0CF83309105AD
:1023F00008F0C7CEFC01EE0FFF1FED5AFE4F019013
:10240000F081E02D89E090E080CF82E190E0E8E982
:10241000F2E07BCF8091E702811509F45BCF853034
:1024200009F458CF8091E80083FD54CF8091E800F3
:1024300082FD7FCF8091E80080FF75CF9091F300FF
:102440008091F2002115310519F08830910550F086
:1024500041E0089709F040E08091E8008E77809392
:10246000E80061CF44914093F10031962150310949
:102470000196E8CF803809F084CE8091E800877F0C
:102480008093E800809116028093F10070CE811154
:1024900078CE10911A02123008F073CE8091E800C5
:1024A000877F8093E800109316029CDA1115D9F00B
:1024B00084E08093E70242E061EC81E029DB42E2C4
:1024C00061EC84E025DB42E261EC82E021DB42E268
:1024D00060EC83E01DDB8091E702843051F482E000
:1024E000809315014ECE8091E30087FDE1CF81E01E
:1024F000E0CF81E0F5CF811509F445C0823849F479
:1025000036D881FF40C089E395D8ABDC89E3ABD8EE
:10251000A8CC833841F42BD880FF35C083E58AD816
:10252000A0DC83E5F4CF843841F421D882FF2BC0AE
:1025300087E480D896DC87E4EACF9CEF980F913A45
:1025400030F390E2980F983050F4877091E001C01A
:10255000990F8A95EAF7892F0E94E504D9CF9BE568
:10256000980F933018F480E090E014C898E5980F25
:102570009B3118F480E090E035C893E3980F9331D5
:1025800010F460E0DDC80895811531F09091AF033B
:10259000892B8093AF0365CC0895811519F00E94B3
:1025A000E5045FCC0895811531F09091B303892B38
:1025B0008093B30356CC0895811539F0809590919E
:1025C000B30389238093B3034CCC089580919D037A
:1025D000811521F082E2F0DF10929D0308950F93A0
:1025E000CF93DF93C5EAD3E0488159816A817B812B
:1025F00088E090E00E94E033288139814A815B8144
:102600006C817D818E819F8100E20E94FA32622F6F
:1026100083E290E00E94CE33DF91CF910F91089535
:10262000E5EAF3E085E0808311828FEF8283838384
:102630001482CF01D4CF8091A903833018F48F5F27
:102640008093A90385EA93E0CACF8091A9038115FD
:1026500019F081508093A90385EA93E0C0CFA0E0F0
:10266000B0E0E5E3F3E10C945332182FF62E042F7B
:10267000E22E9091A50390FF23C0E92FE695E69501
:10268000AE2FB0E0A75ABE4F8C918093A3039C7FDE
:102690009430D9F4612F7F2D842F0E940307962F49
:1026A000672F482F892F0E94BB071093A603F09233
:1026B000A7030093A803E11419F085EA93E08FDFE4
:1026C000CDB7DEB7EBE00C946F32823019F4009195
:1026D000A803EBCF863019F41091A603E6CF89301A
:1026E000D9F3893111F7E9512E2F2170922EE695F9
:1026F000F0E0E05FFA4FE491CE2FD0E0A12CB12CB6
:10270000C12CD12CC50124E0969587952A95E1F737
:10271000911012C0810F9601402F6F2D0E948A07E1
:102720008FEFC81AD80AAC0EBD1E20E1C216D10424
:1027300049F70E94A607B9CF212F281B822FEBCF84
:10274000E5EAF3E0818121E043816281885F87CF00
:10275000E5EAF3E0818121E04381628188507FCF07
:10276000E5EAF3E0628128E0620F08F46FEF21E010
:102770004381818174CFE5EAF3E0628128E0621B46
:1027800008F460E021E04381818169CFE5EAF3E06C
:10279000438128E0420F08F44FEF21E062818181FC
:1027A0005ECFE5EAF3E0438128E0421B08F440E015
:1027B00021E06281818153CFAFE0B0E0E2EEF3E14E
:1027C0000C944F32FE0131968AE0DF011D928A950A
:1027D000E9F784E8E82E81E0F82E8F0199E8C92E08
:1027E00091E0D92E3F01AA24A394B12C30E9832E85
:1027F00031E0932EF70181917F018F3F09F43EC0B4
:10280000F894E82FE295EF70F0E021A18F70A50118
:1028100002C0440F551F8A95E2F7CA01922F982BE8
:1028200091A392A18095892382A3789400C0E9E8BE
:10283000F1E031E0512C21912F3F79F0A22FA295A8
:10284000AF70A05EB0E08C9190E02F7002C09595C3
:1028500087952A95E2F780FF73C080E0582A330FEE
:102860008E169F0641F7F70182918F3F11F00E946B
:10287000E90650EA5A95F1F7D8015C920F5F1F4FB5
:10288000CE14DF0409F0B6CF4AE050E0B30182EB8A
:1028900092E00E9480339C01892B41F08AE0F30191
:1028A000A2EBB2E001900D928A95E1F70091BD0292
:1028B00010E005521D4F232B09F444C081E08093A2
:1028C00011020E94420B9093100280930F0280919C
:1028D0000303811509F490C07E01BBE0EB0EF11CEF
:1028E00085E0F70111928A95E9F7809112028A300A
:1028F00008F04CC041E955E1B701C8013ADA811549
:1029000009F468C046E355E1B701C80132DA811520
:1029100009F460C0109212028091BC0290E045E080
:1029200050E0B70185529D4F0E94803321E02093F3
:102930000E02892B09F041C02F96EFE00C946B3208
:10294000832F8CCF80911102811509F4C0CFE090C4
:102950000F02F09010020E94420B8E199F090597FA
:1029600008F4B5CF45E050E062EB72E0C8010E9488
:102970008033892B41F085E0E2EBF2E0D801019051
:102980000D928A95E1F710921102A1CFC0900C022E
:10299000D0900D020E94420B8C199D09843F9140FA
:1029A00008F0A8CF80910E02811531F285E0D701A1
:1029B0001D928A95E9F710920E02A091BC02B0E038
:1029C000A552BD4F85E0FE013B9601900D928A9580
:1029D000E1F7B2CF809112028F3F39F40E94420B8F
:1029E00090930D0280930C02DDCF8F5F80931202D3
:1029F0008A3008F491CFF2CF85E0F801ADEEB2E075
:102A000001900D928A95E1F78DEE92E068D880935F
:102A1000EC02C090F202D090F302E090F402F09049
:102A2000F5028091080290910902A0910A02B091EA
:102A30000B02C816D906EA06FB0609F47DCFC09240
:102A40000802D0920902E0920A02F0920B020E9460
:102A50005B0CC61AD70AE80AF90AC092FF02D092A4
:102A60000003E0920103F092020366CFCF92DF925F
:102A7000EF92FF921F93CF93DF9300D000D0CDB79A
:102A8000DEB7C090E802D090E902E090EA02F09050
:102A9000EB020E945B0C6C197D098E099F0911E005
:102AA000643671058105910578F10E94670CDC019F
:102AB000CB010296A11DB11D89839A83AB83BC8390
:102AC000809134019091350184519D4F20913301C3
:102AD000422F50E0253010F044E050E0BE016F5F1F
:102AE0007F4F0E948D3382E090E00E94DE31182FEC
:102AF000811551F00E945B0C6093E8027093E9022B
:102B00008093EA029093EB02812F0F900F900F9029
:102B10000F90DF91CF911F91FF90EF90DF90CF90BA
:102B200008958F929F92AF92BF92FF920F931F933F
:102B3000CF93DF9300D000D000D0CDB7DEB7F62E14
:102B4000072F80E090E00E94DE31182F811509F4F4
:102B500060C080912601482F50E0811511F041E0BE
:102B600050E0609127017091280164517D4FCE01A2
:102B700006960E948D338090FB029090FC02A090FC
:102B8000FD02B090FE020E945B0C681979098A0967
:102B90009B09643671058105910538F48DEE92E04C
:102BA0000E946F0D9E818917A1F181E090E00E9443
:102BB000DE318115C9F180912E01482F50E0863019
:102BC00010F045E050E060912F01709130016451A8
:102BD0007D4FCE0101960E948D338DEE92E00E94D2
:102BE0006F0D9E81891320C00E945B0C6093FB02D5
:102BF0007093FC028093FD029093FE0285E0FE013B
:102C00003196A6EFB2E001900D928A95E1F781E04E
:102C10000CC085E0EDEEF2E0DE01119601900D9220
:102C20008A95E1F71111EACF80E095E0E6EFF2E056
:102C3000AF2DB02F01900D929A95E1F70F900F9064
:102C40000F900F900F900F90DF91CF911F910F91E8
:102C5000FF90BF90AF909F908F9008950F931F9318
:102C6000CF93DF93833030F56A3020F5473010F58D
:102C7000C42FD0E0CC0FDD1F2EE0629FC00DD11D10
:102C800011243CE8839FC00DD11D1124CE018996EB
:102C90000E94AD33082F10E0102F0027CE018A9636
:102CA0000E94AD339801282BC901DF91CF911F916C
:102CB0000F91089580E090E0F8CF462F672F209184
:102CC000070330910803232B81F4703F39F4403F10
:102CD00061F4809105039091060308957A3028F4F9
:102CE000473018F4833008F4B9CF80E090E00895BD
:102CF000A0E0B0E0EEE7F6E10C9457327C010091E1
:102D0000B2038091B103082BC2E0D0E010E0C8010B
:102D10000C2E02C0959587950A94E2F780FD09C0B4
:102D20002197A8F7D12C8D2DCDB7DEB7E7E00C9415
:102D30007332DC2EB7018C2FC0DF0E94EB050197A8
:102D400079F3F1CF0F931F93CF93FC018781908587
:102D5000009789F4858100811181811581F06115C9
:102D600071F0C801C5DFC82F682FC8010E94370461
:102D7000B8018C2FA2DFCF911F910F910895C80148
:102D80000E946D04C82FF4CFCF93DF93D82FC92FA3
:102D9000AFDF6D2F7C2F91DF0E94EB05DF91CF918C
:102DA0000895FC0184818115B1F087819085009799
:102DB000A1F00E94EB05282F92959F709630B9F0F4
:102DC00080F4925F9F70923030F4203FD1F058F43D
:102DD00081E0283E58F080E0089580819181D4DF21
:102DE000EACF9A5FEFCF81E0243FA9F7089591E001
:102DF000813F09F090E081E0283E08F080E0892BD7
:102E0000089581E00895382F292FCB01A32FB22FE9
:102E1000833022E09207A105B10520F483509E4F34
:102E20000C94AD3380E0089585E290E00E94AD33CC
:102E3000893E89F486E290E00E94AD33893059F4EE
:102E400087E290E00E94AD3391E0893409F090E090
:102E5000892F8170089580E0FCCFA6E0B0E0E3E325
:102E6000F7E10C94573207E413E08DECE82EFF24D1
:102E7000F39498E0D92E46E050E0B701CE010196D8
:102E80000E949D33F8018D2D11928A95E9F7B801C2
:102E90006C5F7F4F89819A810E949509F801918327
:102EA0008083B8016B5F7F4F8B819C810E94950965
:102EB000F801938382838D8186838E818783F6E0F8
:102EC000EF0EF11C085F1F4F8DEFE81681E0F8064A
:102ED00091F62696E7E00C947332A6E0B0E0E3E7C3
:102EE000F7E10C945132A090E502B090E60281E047
:102EF00090E09093E6028093E502812C912C10E003
:102F0000640100E01AC021E030E0123021F0F70146
:102F1000859195919C01472D602F812F0E940A0F6A
:102F2000739422E0E20EF11C37E07312ECCF0F5FD6
:102F300087E0C80ED11C0A3049F0C601880F991FDE
:102F4000DC01A850BD4F7D01712CDDCF1F5FB6E4C1
:102F50008B0E911C1330A1F6FE01319686E0DF0145
:102F60001D928A95E9F70DEC11E07F0146E050E0F3
:102F7000B801C7010E94EC330A5F1F4F0D3FB1E05B
:102F80001B07A1F7B092E602A092E5022696EDE0BB
:102F90000C946D32A0E0B0E0E0EDF7E10C9450321B
:102FA000FC018280648081E08483E0E1F4E094901D
:102FB000EFE8F4E0E4910091A8030695015810E0D1
:102FC000000F111F012F1127C0E6D2E0C12CD12C18
:102FD000AA24AA94B12C77247A94E919EE2EF12C24
:102FE00083E0881630F48091A60388838091A7033C
:102FF0008983611017C01B821A8296014A816981F8
:1030000088810E948A078FEFC81AD80A259680E126
:10301000C816D10429F70E94A607CDB7DEB7EEE0A7
:103020000C946C328B818115E9F081508B83789EF2
:10303000C00111246C8170E00E948F32FB01FF27D8
:10304000E05FFB4F8491E82FE9197E9EC0011124B7
:10305000B7010E948F328091A803689FB0011124AC
:103060007A83CBCF0E945C33B5010E94A3328017D4
:1030700091071CF683E0881688F00E945C33B50146
:103080000E94A33288830E945C332091A703269577
:10309000622F70E00E94A332280F29831A82809148
:1030A000A803893C20F088EC8C838B83A6CF8431E5
:1030B000D8F784E1F9CF9091A50390FF2CC081153A
:1030C00059F18B3258F58F73880F880F9091A503B3
:1030D0009370892B8093A503611519F085EA93E01D
:1030E0007EDA6091A5036695669570E04BE050E04E
:1030F00087E091E00E947333892B91F01092A40332
:1031000081E08093CF0220E04091A8036091A70363
:103110008091A603A4CA089581E0D6CF8AE2D4CFD5
:1031200081E08093A4030E947F0C9093CD02809352
:10313000CC02E6CF8091A503869586958F5F8B3272
:1031400008F081E061E0B7CF8091A5038695869570
:103150008A9509F48AE261E0AECFA0E1B0E0E3EB4A
:10316000F8E10C944E32FE01319680E1DF011D92B0
:103170008A95E9F701E210E09DEFA92EBB24B394F4
:1031800023E0422E22E0522E612C712C4F0173015C
:103190006201B1E14B165104610471041CF080E13D
:1031A000C82ED12CA601B501C4010E94BF33AC0CBE
:1031B000BD1C0D2C000CEE08FF084C185D086E08B5
:1031C0007F080150104019F76096E0E10C946A32D4
:1031D0006FEF85E290E00E94CE336FEF86E290E0E1
:1031E0000E94CE336FEF87E290E00E94CE3360E022
:1031F00088E290E00E94CE3370DEAFDF69EE85E2B8
:1032000090E00E94CE3369E086E290E00E94CE33E7
:1032100069E487E290E00C94CE3363EE7EEF80E0C9
:1032200090E00E94E83360E082E090E00E94CE33BC
:1032300081E08093B10361E083E090E00E94CE33AF
:1032400060E074E184E090E00E94E833E9D9C0DFF7
:1032500040E050E0BA018FE090E00E94E03340E0AF
:1032600050E0BA0183E190E00C94E033982F8B3268
:1032700058F4853098F0EBEFE80FE63278F4F0E0A0
:10328000E158FB4C0C94B632833450F48A3308F086
:1032900060C0853339F081E0983309F080E008950B
:1032A0008334E1F781E00E9419040E94800F01C07D
:1032B000B4DF81E008958091C102807F8093C102D4
:1032C00081E080933303F5CF8091E5029091E6028F
:1032D000892B79F30E94800F2FEF84E39CE021502B
:1032E00080409040E1F700C000000E94870C909160
:1032F000C102892F8E7F90FF81608093C10280FD83
:10330000D8CF817F8093C102D4CF9091C102892F01
:103310008D7F91FF82608093C10281FFCACF80912F
:10332000C1028160EFCF9091C102892F8B7F92FF04
:1033300084608093C10282FDF2CFBBCF9091C10225
:10334000892F877F93FF88608093C10283FDE7CF39
:10335000B0CF995381E001C0880F9A95EAF7A3CFC7
:103360009D51F8CFCF93C82F8115C9F08238C9F489
:103370000E94B70A81FD13C089E30E941A0B0E94C4
:10338000310F2FEF37EE83E0215030408040E1F7DE
:1033900000C0000089E30E94330B0E94310FCF91DF
:1033A00008958338A1F40E94B70A80FDF8CF83E521
:1033B0000E941A0B0E94310F9FEF21EE34E09150D2
:1033C00020403040E1F700C0000083E5E4CF8438BE
:1033D000A1F40E94B70A82FDE2CF87E40E941A0B93
:1033E0000E94310F8FEF91EE24E0815090402040F9
:1033F000E1F700C0000087E4CECF8CEF8C0F813A5C
:1034000008F0B3C0809133038130D1F0823089F16C
:1034100081112CC08091AF03823221F48C2F26DFE2
:103420008111BDCFE2E0F2E08191C81709F4D1C06B
:1034300082E0E830F807C1F78C2F0E941A0BADCF5D
:103440008091AF03823251F3C43181F048F4CB3024
:1034500009F4A5CFC03131F782E0809333039FCFC9
:10346000C93221F0C83309F49ACFDCCF109233036C
:10347000D9CFCF3409F46FC0C0F4C832A0F4CE3134
:1034800098F5C73009F454C0C43109F088CF809151
:103490003203811509F483CF109232031092310365
:1034A000109230037CCFC932F0CFC13509F455C03A
:1034B000C23509F454C086EFC03509F070CFE091F1
:1034C0003003F0913103309709F469CF2081082E41
:1034D000000C990B820F911D811531E093070CF4BC
:1034E00040C08FEF80835BCFCD51C0933203C43097
:1034F000C9F078F48FE391E0C23031F080E491E0DC
:10350000C33011F48EE391E0909331038093300344
:1035100046CFC53051F08BE391E0C630A9F310924D
:1035200032033DCF8DE391E0EFCF8CE391E0ECCF20
:1035300081E08093400184E180933F018AE08093A1
:103540003E018EE180933D0188E080933C0188E25A
:1035500080933B0124CF8AE0B2CF8FEFB0CF81E0E0
:10356000AECF97FFBFCF10821ACF80E28C0F88308A
:1035700068F4C77021E030E001C0220FCA95EAF775
:103580008091AF03822B8093AF0307CF8BE58C0F25
:10359000833038F42C2F2452330BC9010E94CA0AFD
:1035A000FECEE8E5EC0FEB3150F4F0E0EE0FFF1F3C
:1035B000E853FE4F808191810E94F20AF0CE83E3AE
:1035C0008C0F833108F0EBCE61E08C2F0E94A00BB2
:1035D000E6CE8C2F0E94330B0E94310F2DCF1F930C
:1035E000CF93DF93182FEB01BDDE209739F4812FA5
:1035F0000E947B12DF91CF911F9108958FE99FE088
:103600000197F1F700C000002197EFCFEF92FF92F2
:103610000F931F93CF93DF93C62FD42F122F8115B3
:10362000A9F06093A1030E94420B9093140280932F
:103630001302C77081E001C0880FCA95EAF70E94A3
:10364000C412CDB7DEB7E6E00C9474328091A103CA
:10365000681333C0E0901302F09014020E94420BF2
:103660008E199F09883C910540F500E20D0FCD179A
:10367000A9F0C770FF24F3948F2D01C0880FCA955D
:10368000EAF70E94CD12083048F48D2F877001C0F0
:10369000FF0C8A95EAF78F2D0E94C41260E070E05B
:1036A000812F9DDF083068F6D77081E001C0880F58
:1036B000DA95EAF70E94CD12C4CFC77081E001C04D
:1036C000880FCA95EAF7F6CFA0E0B0E0EAE6FBE1A2
:1036D0000C945532EC018881811511F1813009F08B
:1036E00046C08981813051F48A81239660E570E07B
:1036F000893311F060E070E072DFEDCF823021F4A9
:103700008A8123962FDEE7CF833029F48A8123969E
:103710000E947B12E0CF843041F022968111DBCFF2
:10372000CDB7DEB7E9E00C9471328A81239620E0B0
:1037300030E09AE0682F6053770BAB016A30710577
:1037400060F02115310551F3EFE9FFE03197F1F712
:1037500000C0000021503109F4CF929FB001939F27
:10376000700D11249A01260F371F8991E3CFE82F9E
:10377000F0E0E354FE4FB490282F26952695269529
:1037800030E0F901E355FE4FE4908770F12C082EEC
:1037900002C0F594E7940A94E2F7E0FAEE24FF24DD
:1037A000E0F8F901E356FE4FC490D12C082E02C078
:1037B000D594C7940A94E2F7C0FACC24DD24C0F86B
:1037C000F901E357FE4F049110E002C015950795EB
:1037D0008A95E2F701701127E114F10411F081EEEE
:1037E000C1DDC114D10411F086EEBCDD60E070E0F3
:1037F0008B2DF5DEC114D10419F086EE0E947B12E8
:10380000E114F10419F081EE0E947B1201151105FB
:1038100021F060E070E08CE2E2DE21965CCFA9E06E
:10382000B0E0E5E1FCE10C944C328C01DC01149633
:103830008C91811509F4C2C061E0C80183DA7C0172
:1038400080919C03811136C0F8018581811509F4AE
:1038500069C0E114F0E5FF0608F04EC0E11420E273
:10386000F20608F0AFC0E11437E0F30619F1F0F406
:10387000C701805E91090897E8F03091AF0380910D
:10388000B3032091AE0399E0F801A8E8B3E00190FA
:103890000D929A95E1F7F0929003E0928F031092C7
:1038A0009203832B822B8093870304C0E1145FE093
:1038B000F50619F7D80115964C91411185C123E7FA
:1038C000E2162CE7F20609F469C0A2EAEA16A2E5BC
:1038D000FA0609F491C208F066C2C7019052811538
:1038E000904208F47BC2B1EEEB16F10409F484C2F5
:1038F000E5EEEE16F1045BC290EEE91692E5F906EC
:1039000050F4A0E6EA16A2E5FA06A0F6C701925521
:1039100080349105B1CF970127573C4725303105B9
:1039200008F0ABCFF9E7EF16FCE7FF0609F04EC051
:1039300020918F0330919003232B81F18115A1F009
:1039400081E00E94910A809187030E94D31289E04E
:10395000E8E8F3E0AEE3B3E001900D928A95E1F779
:103960008091920380933D0386E0F801AEE3B3E0DB
:1039700001900D928A95E1F780913D0380939C031D
:103980008EE393E04CDF10929C03D80115968C9146
:10399000811104C0809187030E94DC128091B403DE
:1039A0008770811559F0F8018581811539F0809172
:1039B0000D0482FF03C082E00E94CA042996E2E15E
:1039C0000C946832F8018681803156CFBAE7EB1645
:1039D000BCE7FB0609F06ECF811509F4CAC0A090C0
:1039E0008F03B0909003E0918703E887E983BE01DD
:1039F0006F5F7F4FC5010E9495092C01F981F987FE
:103A0000F7E4CF2EF3E0DF2EEE24E394F12C222412
:103A10002A94D60117963C90179733FE54C06D90A8
:103A20007C90119712968D909C9013974614570492
:103A3000B9F41496BC91BF83232DF60146816B2FF8
:103A400089850E94AF09811559F08F810E94030476
:103A5000281634F4D60115969C917401F92A282E63
:103A600048145904C9F431FE17C0F601F581FF83EB
:103A7000232DD60116964C916F2F89850E94AF0990
:103A8000811551F08F810E94030428162CF4F60151
:103A900094817301F92A282E30FE15C0FFEF2F12F2
:103AA00012C021E0E216F10471F4232DD60116961E
:103AB0004C9160E089850E94AF09811521F0F601E3
:103AC00085817401F82AF8E0CF0ED11C27E833E095
:103AD0002C153D0509F09DCF31E0E316F104F1F519
:103AE000988592959F704885942B9F7081E0403116
:103AF00008F480E0F82EF294E0EFFE22F92AA114F7
:103B000050E2B50620F5A11481E0B80608F055C0D2
:103B1000EA2C8F2D8D704A2D811509F451C06AE071
:103B200088E697E00E94A20A282F30E0211531058F
:103B300051F44E2D6EE182E497E00E94A20A282FF4
:103B400030E0811549F0F901FF297F0107C0C50167
:103B500090528115904390F1E12CF12C87E0E3E93C
:103B6000F3E0DF011D928A95E9F7F0929B03E09262
:103B70009A0380919A0390919B03892B09F40ECFAD
:103B8000F8018581811539F08FEF0E94910A8091AB
:103B900092038093910386E0F801A3E9B3E00190DA
:103BA0000D928A95E1F78091910380939C0383E9BC
:103BB00093E035DE10929C03F1CEFB28BB24A8CF06
:103BC00068E080E697E0AECFC7019757803891054F
:103BD00008F0FAC6BE2CF0E1EF1608F0DFCE62E086
:103BE00072E080E090E00FD98111D8CEC12CD12CA9
:103BF0007601B11042C074E0272EAE014F5F5F4FD7
:103C00005E834D83AD81BE81E22D1D92EA95E9F779
:103C100046015701FFEF8F1A9F0AAF0ABF0AC7017B
:103C2000B601F1D88983811509F4B8CE813009F045
:103C3000A6C02601370122E0420E511C611C711CF6
:103C4000C501B401E0D8382E8A83811509F4A6CEC7
:103C50008FEF830D833028F5C301B201D4D88B8355
:103C6000811519F0CE0101962FDD4601570133E091
:103C7000830E911CA11CB11C4BC023E0C21622E094
:103C8000D206E104F10409F489CEC701B601BBD81C
:103C90003FEFC31AD30AE30AF30A8111EECFBA94B5
:103CA000A8CF8BEF830D8330B0F54601570143E079
:103CB000840E911CA11CB11CC301B201A4D88B833A
:103CC000811531F1C501B4019ED88C838115C9F0ED
:103CD000AB80BC8051E0A5165FEFB50610F0BA2CA2
:103CE000AA2486E0381651F097E0391619F0C5017C
:103CF0000E945127C5010E94832703C0C5010E946D
:103D000051274601570154E0850E911CA11CB11C9E
:103D10007501640177CFA4E0530142013A12F8CF54
:103D2000C301B20170D8782E46015701B4E08B0E62
:103D3000911CA11CB11CC701B6016D5F7F4F8F4F55
:103D40009F4F61D8711409F429CE811509F426CE4C
:103D50008150990B4FEF489F9001499F300D1124DE
:103D6000E72DE150FF0B2E0F3F1F2150310980F24C
:103D70008FE99FE00197F1F700C00000F6CFCE0178
:103D80000196A2DCC5CF1092AF030E94ED040E9401
:103D9000420B88579C4E90939F0380939E0381E033
:103DA00080939D03FBCDF2EBEF16F2E5FF06E9F5FC
:103DB00025EE30E02770332781E090E001C0880FC6
:103DC0002A95EAF72091A00330919D033115E1F087
:103DD0004115A9F0282B2093A003E0CDD801169619
:103DE0008C91803110F58F2D99278F719927823012
:103DF000910511F04297DBCF21EE30E0DBCF8095CB
:103E000082238093A003CACD322F3823311569F065
:103E1000982F909592239093A0030E94E504D801D7
:103E200015968C91811509F4B9CD80919D0381156A
:103E300009F4D1C0C090AF03D090AE030E94420BF2
:103E400088579C4E90939F0380939E03F801858131
:103E5000811509F4C0C08D2D8C298D79811190C0F8
:103E6000E114F0E5FF0608F5E11420E4F20608F09D
:103E70009BC036EEE316F10409F449C0C701905225
:103E80008115904208F097C0D80116968C91803128
:103E900008F46EC0C70199271092B3038D329105C3
:103EA00009F582E08093B3038AC0B0EEEB16B2E569
:103EB000FB0608F04DC0E0ECEE16E2E5FE0638F534
:103EC000F0EAEF16F2E5FF06E8F420E6E21622E556
:103ED000F206E8F4C701925580349105C0F01092C3
:103EE000B303C7018E32910508F082C08832910574
:103EF00008F063C08E31910508F061C004974A97BD
:103F000080F23EC034EBE31632E5F30641F7D80108
:103F100015969C91911509F42FC51092A103970154
:103F200030572332310508F036C584E090E00E9416
:103F3000BA3390930D0480930C04F701E150F047DD
:103F4000E232F10508F076C0EB55FB4C0C94B6322A
:103F500049E7E4164CE7F40630F457E7E5165CE76A
:103F6000F506A8F6BCCF8BE7E8168CE7F806CECFAF
:103F70008F2D8F71843159F2863161F41092B30321
:103F80000E94E6128091AF039091A003892B809349
:103F9000AF0321C00E94E6128091AF039091A0036D
:103FA000892B8093AF03B3CFD80116968C918031C3
:103FB00008F070CFACCFC7016FCF8A9709F7809117
:103FC000A003811531F08091B30392E0892780939B
:103FD000B3030E94310FF8018581F701E851FC47D6
:103FE000E730F10508F093CFE953FB4C0C94B6325F
:103FF0008C34910521F38D329240E0CF26E241EEE0
:1040000061EE04DBCBCC27E245EE65EEFACF26E28B
:1040100041EE60EEF6CF27E245EE64EEF2CF26E207
:1040200041EE62EEEECF27E245EE66EEEACF28E201
:1040300041E0EBCF80910C04816080930C0460918F
:104040000C0470910D0484E090E00E94E8330E941B
:10405000800FA4CC80910D04886080930D04EFCF75
:1040600080910C048260E9CF80910C048460E5CFDC
:1040700080910C048860E1CF80910D048160EDCFC8
:1040800080910D048260E9CF80910C048061D5CFCE
:1040900080910C048062D1CF80910C048064CDCFDC
:1040A0000E94800F80910C048068C7CF80910C041F
:1040B0008C60C3CF80910D048360CFCF80910C04BE
:1040C0008E7FBBCF80910D04877FC7CF80910C047A
:1040D0008D7FB3CF80910C048B7FAFCF80910C0488
:1040E000877FABCF80910D048E7FB7CF80910D0479
:1040F0008D7FB3CF80910C048F7E9FCF80910C0475
:104100008F7D9BCF80910C048F7B97CF0E94800F77
:1041100080910C048F7791CF80910C04837F8DCF99
:1041200080910D048C7F99CF80910C04992782FF98
:10413000939590FB82F990FB83F97FCF80910D04DA
:10414000982F909590FB80F990FB81F986CF909104
:104150000C04892F8F7B96FF80646FCF0E94800FA5
:1041600090910C04892F97FB87F9805866CF61E006
:104170008EE090E00E94CE3362CF60E0F9CF909164
:104180000C04892F8F7E94FF806157CF90910C048F
:10419000892F8E7F90FF816050CF90910D04892FE1
:1041A000877F93FF886059CF89E208C489E2F0C312
:1041B000B7E7EB16BCE7FB0609F060C081E00E94A0
:1041C000290480C08272F701E052F847EB30F10514
:1041D00008F04FC0E253FB4C0C94B6328091A5031B
:1041E00080FF0CC08E7F8093A50385EA93E00E9438
:1041F000EF121092A4030E94A607D0CB8160809397
:10420000A50361E0869586950E945B18C7CB811552
:1042100029F00E94A418C2CB8115D9F30E949A18E4
:10422000BDCB811529F00E94A813B8CB8115D9F315
:104230000E94A013B3CB811529F00E94BB13AECB13
:104240008115D9F30E94B013A9CB811529F00E94E2
:10425000D113A4CB8115D9F30E94C6139FCB81152E
:1042600029F00E9425139ACB8115D9F30E941B13C4
:1042700095CBE7E7EE16ECE7FE0609F1F8E7EF1657
:10428000FCE7FF0629F19701205E32452032310517
:1042900020F5911122C02E2D2F7181E090E0AC010C
:1042A00002C0440F551F2A95E2F77A01642F83E07C
:1042B00090E00E94CE338E2D0E9419046FCB81E0D6
:1042C0000E941F0443E062E081E00E94A10466CBEB
:1042D00082E0911509F473CFF3CF4091AD03809143
:1042E000B203282F30E02095309570E02423372347
:1042F000232B19F048234093AD035BE7E5165CE7F9
:10430000F50641F4911509F449CB0E9406040E9478
:10431000DD0944CB80E4E81682E5F80608F05AC0CF
:10432000A0E2EA16A2E5FA0608F05BC0E114B0E5E7
:10433000FB0670F5E114E0E4FE0608F068C0911594
:1043400009F47EC0BAE5EB16BCE7FB0609F4DAC057
:1043500008F0BCC0F1E0EF16FCE7FF0609F4D0C09E
:1043600023E0E2162CE7F20609F4C4C0E1143CE7AE
:10437000F30609F065C00E94800F8FEF94E3ACE074
:1043800081509040A040E1F700C000000E94870CDF
:10439000970130552115324090F6970145E036954A
:1043A00027954A95E1F7822F8F702091AD0330E079
:1043B00041E050E0082E02C0440F551F0A94E2F776
:1043C00024233523232B09F4BACF9111A0CF1092C7
:1043D000AF03F6C29701205C32452032310508F068
:1043E000AECF8E2D8F712091AD0330E041E050E0D3
:1043F000082E02C0440F551F0A94E2F724233523E8
:10440000232B09F49CCF911509F4C8CA80CFD80199
:1044100016968C91803108F092CF911111C02F2DFA
:104420002F7081E090E002C0880F991F2A95E2F773
:104430002091AD0330E082239323892B09F0AECA8B
:10444000D80117968D919C91009709F45FC00E9446
:10445000EB057C01D8011596BC9015971696AC908B
:10446000A2942FE0A2228091B4038770811509F1F4
:10447000CB2CB114F9F08F2D807F803469F080E26D
:104480008E0D8830B0F08F2D807E803229F4B2E01E
:10449000EB1678F0A11469F080910D0482FF09C039
:1044A00082E00E94CA048091B4038770CC24C39434
:1044B0008111C12CEF2DE295EF70F0ECFF1608F0A2
:1044C0009FC0F0E0E752FB4C0C94B6324BE5E4168B
:1044D0004CE7F406C9F080910D04002482FF039498
:1044E000802D5CE5E5165CE7F50609F0A9CF0E9492
:1044F000F30EA6CF6FEF7FEF80E090E00E94E833ED
:104500000E94A30F81E0F3CF80E0F1CFF801858115
:10451000C080D180811569F0C6010E947816F82EFE
:10452000682FC6010E943704B6018F2D0E945D16C8
:104530008ECFC6010E946D04F82EF6CF2F2D2F705E
:10454000D22E30E1F31618F0D29490EFD922B114A4
:10455000B9F0D11469F080E28E0D883010F0E110CE
:1045600009C08091AF038D298093AF030E94310F62
:104570008E2D44C08091B3038D298093B303F6CF71
:104580008E2D0E947B12D114D9F180E28E0D8830DD
:1045900010F0E11004C08D2D0E94E50406C0D094F7
:1045A0008091B3038D218093B3030E94310F28C003
:1045B0004F2D4F70D42E8F2D807F803219F0D294E2
:1045C00080EFD822E11451F051E0E51609F483C0E0
:1045D000B11409F48FC0A114A9F1CACF80910D04C0
:1045E00082FD2CC0B11421F1D11439F08091AF03B8
:1045F0008D298093AF030E94310F80E00E94B21991
:10460000C11409F4D9C08091B40380FDD5C0F8016C
:1046100015828695869586950E941F04C801FFD84D
:104620008091B4038695869586950E942904C4C01E
:1046300080E00E947B12D11419F3ADCFB11469F15F
:10464000A11004C08D2D0E94C412DACF81E0A812FF
:1046500010C0F090AE038D2D8F21D81689F20E94E4
:10466000420B9093B8038093B703FD28F092AE03FA
:10467000C7CF95E0A912C4CF8D2D0E94C4128D2DF5
:104680000E94620B8091B0039D2D9823D91609F4E6
:10469000B7CF8D298093B003B3CFA11012C08D2D59
:1046A0000E94CD128D2D0E94620B8091B0039D2D32
:1046B0009823911509F4A4CFD094D822D092B003B6
:1046C0009FCFA1E0AA129CCF8091AF038D218115CD
:1046D00009F496CFE4CFB11429F0B6E0AB1608F098
:1046E0008FCFB0CFE5E0AE1608F08ACF8D2D0E94B7
:1046F000CD1286CFA114D1F3F9E3EF1209C02FEF49
:1047000037EE43E0215030404040E1F700C0000068
:104710008E2D0E947B1274CF8F2D86958695837087
:10472000811561F0813009F06BCFC7019370B11032
:1047300002C080E090E00E94F20A62CFC70193704D
:10474000B11002C080E090E00E94CA0A59CF6B2DE0
:104750008E2D0E94A00B54CF8F2D8370811139C0F4
:10476000B11028C04E2D429546954770440F440F16
:104770008E2D8F70042E01C0880F0A94EAF72E2D1B
:104780002071E4FE07C02FE030E001C0220F4A95FF
:10479000EAF720953F2D3695369533703230A1F0EB
:1047A000333081F04091B103313059F0822B8423B2
:1047B0000E9419040E94B70A60E0C8010E94A21674
:1047C000FDC8842B822BF4CF822B9091B1038927D3
:1047D000EFCFB11459F1F0FEEDCF4E2D4295469535
:1047E0004770440F440F8E2D8F70042E01C0880F28
:1047F0000A94EAF72E2D2071E4FE07C02FE030E086
:1048000001C0220F4A95EAF720953F2D369536953F
:104810003370323089F0333069F04091B203313077
:1048200041F0822B84230E941C04C4CF823010F2FA
:10483000D4CF842B822BF7CF822B9091B203892780
:10484000F2CF5F2D5F70F52EB11439F0852F0E94E5
:104850001F048E2D0E94C412ADCF8E2D0E94CD124A
:104860008F2D0E942904A6CF82EFE816A1F193EFC5
:10487000E91680F4A0EFEA16E1F0B1EFEB16A1F033
:10488000B11409F467C0A11409F461C08E2D0E940F
:10489000B21990CFE3EFEE1629F1F4EFEF12F0CF5B
:1048A00080910D0482FD2AC08F2D8F71B114C9F241
:1048B00016C0B11469F025E0A21608F07BCF2F2DA9
:1048C0002F7181E090E001C0880F2A95EAF7B5CFFB
:1048D00036E0A316F2CF8F2D8F71B110C2CF0E9498
:1048E0001F0468CF80E0B11409F49DCF9F2D9F7104
:1048F00081E001C0880F9A95EAF795CFB114C1F015
:104900008091B4038770843049F41092B4031092FC
:10491000B6031092B5038F2D8F71A3CF45E063E0EE
:10492000A41608F047CF8F2D8F710E944E0B42CFF7
:1049300055E0A51640F01092B4031092B603109201
:10494000B50364E0F0CF81E00E94CA0433CF8F2D1D
:104950008F71C5CFA114F9F289E3E81209C09FEF66
:10496000A7EEB3E09150A040B040E1F700C00000D6
:104970008E2D0E947B121ECFB6E1EB16BCE7FB0624
:1049800009F016CC8091A203811509F40FCC85E3C0
:104990000E94330B15C08091AF03E6E1EE16ECE701
:1049A000FE0609F00FCC8A7A91E0811101C090E0F7
:1049B0009093A203811509F4F7CB85E30E941A0BAB
:1049C0000E94310F0C94CE1CF3E7EF16FCE7FF06B4
:1049D00011F00C94651C80919D03811509F4D3C9D5
:1049E0000E94E6120C94CE1C80910904803178F468
:1049F00080910804811559F0E091BA032091B90320
:104A0000309104044091030459E02E1301C008952D
:104A10006E2F70E05E9FF0011124DF01A554BC4FA2
:104A200014968C911497811559F111968C911197C8
:104A3000831326C08C91841323C015968C911597EF
:104A400081111EC012968D919C91A0910504B09188
:104A500006048A1B9B0B883C910590F48091090405
:104A60008F70806180930904EF53FC4F80818F70B9
:104A70008061808383E094E00E940F1C0C94C0044A
:104A8000FB013196E770C1CFAFE0B0E0EAE4F5E2B8
:104A90000C9450328C0186E0F801DE011A960190E8
:104AA0000D928A95E1F7F801F580848193E0892ED3
:104AB00094E0992E60900704611017C0811591F061
:104AC000F11409F417C1C8010E94D116811509F427
:104AD00011C189E0F801A3E0B4E001900D928A953C
:104AE000E1F782DFFF24F39456C07080A280B38088
:104AF000D09008042091050430910604A501421BC2
:104B0000530BD11409F4C6C0483C510508F079C0D4
:104B1000811541F380910404C180E090090450E1C3
:104B2000E51608F059C0C81215C08091030487111A
:104B300011C0F1104BC08E2D8F70806180930904DD
:104B400083E094E00E940F1C80910904F8018683A1
:104B5000F12C21C0F1103AC040E06C2D872D0E944D
:104B6000120E40E06C2D872D0E94120EF82E81113E
:104B7000EFCF8A859B850E94C416292F22952F701E
:104B8000903470F49F702230A0F09115B1F0F801CC
:104B90009681903190F48F2D2F96EEE00C946C322C
:104BA0002A5F2F70223068F0C8010E940F1CFD2C74
:104BB000F2CF911511F0811571F3805E883058F3B2
:104BC000F3CF803F40F3815F8330F9CF80910904B8
:104BD000816080930904BCCFC8123BC0809103045C
:104BE000871137C0F11035C0E682C8010E940F1C42
:104BF00089E0F801A3E0B4E001900D928A95E1F715
:104C000071CFE0900904F0E1EF1650F483E094E0F6
:104C10000E940F1C89E0F40111928A95E9F798CF60
:104C2000811509F45FCF90910404F80181819813F4
:104C300010C08091030487110CC0F1100AC0E682F5
:104C4000C8010E940F1C89E0F40111928A95E9F7CE
:104C500049CFC8010E94D116811509F44BC0F11447
:104C600009F448C080910904803208F432CF1E82D2
:104C70001F821886198680910304909104049A83F8
:104C80008983BC82AB826D82EF82CE0101960E9445
:104C90000F1C1FCF483C510508F0BCCF811509F40B
:104CA00021CFF11439F1909104048181981318C037
:104CB00080910304871114C08091090480FD98CF6E
:104CC000803108F495CF8683807F803F09F48DCFB3
:104CD0008681982F907F905F8F70892B868385CFF8
:104CE000C8010E94D1168111F4CE8091090481601F
:104CF00080930904C8010E940F1CF4CEA1E2B0E029
:104D0000E4E8F6E20C945A324C8F5D8F6E8F7F8F01
:104D100088A3192F99A391111092B303198E1A8E9B
:104D20001B8E86E0FE017C96DE01539601900D926B
:104D30008A95E1F708A180910D0482FF1FC00E94AF
:104D4000420B2091B5033091B603821B930B883838
:104D5000934138F08091B40382FD03C082E00E9449
:104D6000CA040E94420B2091B7033091B803821B02
:104D7000930B8838934110F00E94ED04011561F007
:104D80000F8B188F61E0CE0143960E94A21661E05E
:104D9000CE0143960E94A2160F8B188F89E0FE0168
:104DA0007396DE011A9601900D928A95E1F7CE0175
:104DB0000A966ADE811110C02091B9033091BA03BE
:104DC00089E0FE013A96DE01119601900D928A95D6
:104DD000E1F78E8581110BC019E08091BA039091A3
:104DE000B90389132BC0A196E4E00C947632822F8C
:104DF00090E00196877099273817190671F40E9480
:104E0000800F1092B9031092BA0389E0E3E0F4E056
:104E1000DF011D928A95E9F7DFCF99E0929FD001DB
:104E20001124A554BC4FFE01319601900D929A9524
:104E3000E1F78093B9030E94C004CECF189FC00150
:104E4000112485549C4F20DE811569F28091BA03AC
:104E500090E00196877099278093BA03BECFA6E0B1
:104E6000B0E0E5E3F7E20C945A320E94420B8C0169
:104E70008091090390910A038017910771F01982BC
:104E80001A820E94420BBC0149815A8180E090E065
:104E900035DF10930A03009309032696E4E00C948F
:104EA0007632A6E0B0E0E7E5F7E20C945A328C01E6
:104EB0009093060380930503011580E21807B0F470
:104EC000C801805E9109089728F063ED72E1011531
:104ED000110511F464EC72E1C8010E94D703802F20
:104EE0000E94B2192696E4E00C94763280EF898312
:104EF0008A830E94420B8160BC0149815A8181E012
:104F000091E0FCDEEFCFA6E0B0E0E9E8F7E20C9438
:104F10005A328C019093060380930503011580E2B9
:104F20001807B0F4802F0E947B12C801805E91099F
:104F3000089728F06CED72E10115110511F46DEC84
:104F400072E1C8010E94D7032696E4E00C94763201
:104F500080EF89838A830E94420B8160BC01498172
:104F60005A8181E090E0CADEEFCF8F929F92AF929C
:104F7000BF92CF92DF92EF92FF920F93CF93DF9386
:104F800088E090E00E94B5334B015C01C5EAD3E0B4
:104F900068839982AA82BB821C821D821E821F8224
:104FA00083E290E00E94AD33282F30E040E050E0F3
:104FB00060E070E080E090E000E20E94DF322829AB
:104FC00039294A295B29288339834A835B836C8387
:104FD0007D838E839F83DF91CF910F91FF90EF9020
:104FE000DF90CF90BF90AF909F908F900895CDB7F6
:104FF000DEB7AC970FB6F894DEBF0FBECDBF85B756
:10500000806885BF85B7806885BF84B7877F84BF88
:105010000FB6F894A8958091600088618093600035
:10502000109260000FBE80E890E00FB6F894809375
:105030006100909361000FBE81E08093150187EEBF
:1050400096E09093FF018093FE010E942D170E942D
:10505000420D0E94B80D8091E20084608093E200CE
:1050600078948091E702811599F08091E900109180
:10507000EC008F70179511271795182B1092E900E7
:105080008091E80083FD0E94B80F1F701093E90023
:1050900082E084BD93E095BD9AEF97BD80936E004A
:1050A0001092FF021092000310920103109202036B
:1050B0000E941417811102C00E94E8188091D80044
:1050C00080618093D8002AE12A95F1F700C0809191
:1050D000D900182F117080FD04C00E94420D10925B
:1050E000E7021093030310930403109316011111A8
:1050F0000E94F930809116018091160190E0811193
:1051000001C095E09093BD0285E0891B8093BC02AD
:1051100004E811E0E9E8EE2EE1E0FE2ED8018D91E1
:105120008D018F3F11F00E94E906E016F106B1F7FC
:1051300009E811E0F80181918F018F3F11F00E9481
:10514000E906F1E000391F07A9F78AE0EBEDF2E08C
:10515000DF01282F1D922A95E9F7E2EBF2E0DF014B
:105160001D928A95E9F780E090E00E94BA33833E71
:105170009E4F21F40E941417811102C00E940D1944
:1051800082E090E00E94AD338093C10284E090E021
:105190000E94BA3390930D0480930C040E94DC1398
:1051A000EFEFF6E721E0E150F0402040E1F700C0EA
:1051B00000000E94DC138091DB0280FF08C06FEFCB
:1051C0007FEF80E090E00E94E8330E94870C83E04C
:1051D00090E00E94AD330E9419048091BE028111BB
:1051E0001EC085EA93E0C1DE8091A503843028F4D7
:1051F0000E94101385EA93E0B8DE0E94980710928F
:10520000A4030E94D0098091A50380FF05C060E03F
:10521000869586950E945B1881E08093BE028091FE
:105220000303811101C0E8D787E191E090930C035B
:1052300080930B038E010F5F1F4F8091E70270E494
:10524000F72E853009F482C00E94DC1352ECE52E63
:1052500052E0F52E6BEDC62E62E0D62ED601F70198
:1052600091918D912CEC32E02E173F0709F478C014
:105270009817B1F360900303B12CD601AD906D0186
:10528000F70181917F018A1539F1782E7A24912CCA
:1052900088248394872D88218115B9F06114A9F0A1
:1052A0009982BA820E94420B9C838B83F1E0FD833A
:1052B00091E08A2D8821811101C090E09E8349816F
:1052C0005A816B817C818D8119DD9394880C27E054
:1052D0009212E0CFF701A292B3943AE0B312CDCF8D
:1052E0000E94670C40C08091E702843019F110924F
:1052F000BF0288E190E00FB6F894A8958093600013
:105300000FBEF092600083B7817F846083BF83B754
:10531000816083BF7894889583B78E7F83BF0FB6F3
:10532000F894A89580916000886180936000109245
:1053300060000FBE0E94DC13EBEDF2E08191811161
:105340006AC5A5EEB2E0AE17BF07C1F78091E702CC
:10535000853009F4C8CF0E94800F0E94B70A74CF2D
:10536000981388CF7CDD80910303811589F08091AB
:105370009D03811569F00E94420B20919E0330919C
:105380009F03821B930B8F3F9F4710F40E94E612EE
:105390008091A403811509F446C08091A303E09194
:1053A000A503E695E695E81BE093CE02853109F466
:1053B00005C108F0ADC0893009F4F4C008F099C007
:1053C000823009F4D9C0863009F4E1C030EDE32E13
:1053D00037E0F32E42E0C42E47E0D42E8091CF0276
:1053E000811561F01092CF020E947F0C9093CD0244
:1053F0008093CC021092D1021092D0020E947F0CB6
:105400002091CC023091CD02821B930B8F3F9F479E
:1054100050F42E0D3F1D3093CD022093CC028CEC26
:1054200092E0F601099586E0E7E3F3E0D801019008
:105430000D928A95E1F790903803B0903903D0909F
:105440003A03A0903B03C0903C03109239031092A2
:105450003A0310923B0310923C038D2D8B2981154A
:1054600009F4C1C0E090D402F090D5020E94420B32
:105470009C012E193F0990913503911509F4A9C09B
:1054800080913F018217130608F0ADC09F3F19F0CD
:105490009F5F90933503B11459F00E94120A91E076
:1054A0001B140CF09FEF899F802D112480933903EA
:1054B000D11459F00E94120A91E01D140CF09FEFD4
:1054C000899F802D112480933A038091390381159F
:1054D00009F489C0F0903A03F11409F484C00E94E1
:1054E000040A809339038F2D0E94040A80933A03A3
:1054F0007AC08F3009F06ACFE695F0E0E35EF94FAD
:10550000E491EE2EF12CBBE4CB2EB8E0DB2E66CF7F
:1055100064EFE62EFF24F39477E6C72E79E0D72ECA
:10552000843209F45BCFB0F448E2E42EF12C57EE5C
:10553000C52E58E0D52E883109F450CF833209F0BA
:1055400045CFE8E1F6E0E590F590F8EDCF2EF7E0F5
:10555000DF2E44CF853209F039CF8E2F63E0D3D7C9
:10556000E92FF0E0EB5EF94FE491EE2EF12CEAEC3E
:10557000CE2EE7E1DE2E32CFF0E0EA5DF94FE49186
:10558000EE2EF12C22E1C22E28E0D22E27CFF0E021
:10559000ED5DF94FE491EE2EF12C93E0C92E98E0E9
:1055A000D92E1CCFE695F0E0E05EF94FE491EE2EA7
:1055B000F12C85E2C82E88E0D82E10CFF0E0E65E10
:1055C000F94FE491EE2EF12CAFE9CA2EA8E0DA2EC5
:1055D00005CF40914001FAE04F9FA00111244217EE
:1055E000530708F455CF8A2D8C29811509F441C041
:1055F000E090D202F090D3020E94420B9C012E193F
:105600003F0990913403911509F400C42135310507
:1056100080F19F3F19F09F5F90933403A11459F0DC
:105620000E94580A91E01A140CF09FEF899F802D78
:10563000112480933B03C11459F00E94580A91E051
:105640001C140CF09FEF899F802D112480933C0344
:1056500080913B03811569F0F0903C03F11449F00F
:105660000E94040A80933B038F2D0E94040A8093BA
:105670003C0380913803981219C080913903811539
:1056800011F08B1113C020913A03211511F02D1147
:105690000DC090913C03911511F09C1107C0309101
:1056A0003B03311103C0822B892B81110E94770BA0
:1056B00086E0F801A7E3B3E001900D928A95E1F747
:1056C0000E94B70A9091D602891721F08093D602E2
:1056D0000E945B0C8091E702843009F0AECD83E03C
:1056E0008093E9008091E80082FFA7CD8091E800D7
:1056F00090E085FF09C00E94110D30E2E32EF12CED
:105700006801811561F191E08091E8008B778093C9
:10571000E800911509F491CDE0900703F09008039B
:10572000E981E114F10449F1EE3F09F048C08A81B2
:10573000833020F08550833008F041C0EA81EE309C
:1057400008F03DC0F0E0EB51FB4C10C78091F10038
:10575000D6018D936D01B1E0EB1AF108A1F28091B1
:10576000E80085FDF3CF8091E8008B778093E80017
:105770000E94110D811599F3C6CFE43148F4E1156B
:1057800049F0E150E33130F4F0E0ED50FB4CEEC66F
:10579000EE3FA1F28FEF898312C01A8289E08B83DA
:1057A0000EC08A81823079F08330A9F0813091F780
:1057B0000E945B0CF1D66B837C838D839E83C80132
:1057C0000E94610D3ACD88E290E0C7D71B821C820F
:1057D0001D828E83F4CF8091E5029091E602892BA1
:1057E00071F38AE0EBEDF2E0DE01139601900D9289
:1057F0008A95E1F7E4CF8A81823061F66B817C8102
:105800008D819E81C9D688E290E0C8D7D8CF4C81DF
:105810006B818A810E942E169827892798279E835C
:105820008D83CDCF2D813E813227232732274C8196
:105830006B818A810E940A0FC2CF0E946D17BFCF71
:105840008A81823891F1B0F48038E9F0813809F02A
:10585000B6CF60E08B810E945B189B818091A5038D
:1058600091111AC08E7F8093A5031092A4030E9409
:10587000A607A5CF833809F0A2CF20E04091A80366
:105880006C818B8106C020E04B816091A7038091E1
:10589000A6030E942F1393CF81608093A50360E03D
:1058A000869586950E945B188ACF8B818093A90389
:1058B00086CF8A818238E1F060F48038A1F08138A7
:1058C00009F07DCF8091A50380FF10C08695869555
:1058D00066CF833809F073CF8091A6038B838091C4
:1058E000A7038C836CCF8091A80359CF80E057CF5A
:1058F0008091A90354CF0E94980785EA93E00E9403
:10590000EF125DCF80E18A835ACF82E08A8383E001
:1059100046CF8C818D3108F052CF8A809B809824AD
:1059200089249824A12CB12C68017801E80EF11C7F
:10593000CE14DF0409F443CF80E0E3E08E16E2E00A
:105940009E06A104B10420F4C40183509E4F05D7E4
:10595000D60114968C93BFEFCB1ADB0AEFEF8E1AA9
:105960009E0AAE0ABE0AE4CF8091E5029091E6025B
:10597000892B09F424CF8C818D3108F020CF482E5B
:10598000512C612C712CCA80DB80DC24CD24DC24DA
:10599000E12CF12C1801812C912C540184149504D4
:1059A000A604B70408F00BCFF3E0CF16F2E0DF0651
:1059B000E104F10438F4D10114966C91C6018350CE
:1059C0009E4FECD6BFEF8B1A9B0AAB0ABB0AEFEFD8
:1059D000CE1ADE0AEE0AFE0AFFEF2F1A3F0ADECFCA
:1059E0000E94AD18ECCE83E08ECF8C818D3108F013
:1059F000E6CE482E512C612C712CCA80DB80DC2431
:105A0000CD24DC24E12CF12C812C912C54011E019D
:105A100025E0220E311C84149504A604B70408F076
:105A2000CECE80E034EAC31631E0D306E104F104BF
:105A300018F4C601899691D6D1018D931D01BFEF4F
:105A40008B1A9B0AAB0ABB0AEFEFCE1ADE0AEE0AEC
:105A5000FE0AE1CF2C81E22EF12C2D3108F0AFCEE1
:105A60008A819B819827892798272C01612C712C8A
:105A7000843AF1E09F0708F0A2CE822E912CA12C4F
:105A8000B12C44EA51E060E070E044195509660920
:105A90007709421751056105710508F490CE2091F0
:105AA000E5023091E602232B09F03FC09C01275DFF
:105AB0003F4F3CA72BA780FBCC24DD24C0F880FF00
:105AC0000BC088964AD69D818927982789278115FA
:105AD0009C4711F48FEF8D83D501C401840D951D72
:105AE000A61DB71D80FF1AC0170141E0241A310816
:105AF000CE010596820D931D9AA789A78BA59CA51B
:105B00008E0D9F1D2AD6A9A5BAA59C9181159C47EB
:105B100021F48FEFE9A5FAA580837101F801EC0D5E
:105B2000FD1D2FEFCE14DF0428F01801C12CD12C5D
:105B3000760126C09481858181159C4711F42483C8
:105B4000258342E0C40ED11C3296ECCF84EA48167D
:105B500081E058066104710430F4D10114966C910F
:105B6000C20189961BD6BFEFCB1ADB0AEB0AFB0AF0
:105B7000EFEF4E1A5E0A6E0A7E0AFFEF2F1A3F0AF7
:105B8000C814D904EA04FB0408F319CE8091E50295
:105B90009091E602892B09F412CEC8010E94610D92
:105BA0002FEF31EE44E0215030404040E1F700C09B
:105BB00000000BCB88E0E1E4F1E0DE01919601907A
:105BC0000D928A95E1F7FE0132968FE1DF011D9279
:105BD0008A95E9F786E0898388E07F96DE0115964D
:105BE00005CE88E1898381E08A831B821C82E7CD10
:105BF0008B819C81092E000CAA0BBB0B25E0880F22
:105C0000991FAA1FBB1F2A95D1F7AC01BD01405EA9
:105C10005F4F6F4F7F4F481759076A077B0708F49C
:105C2000CECD8831E1E09E07A105B10508F0C7CDD2
:105C30004931F1E05F076105710520F048E151E06D
:105C400060E070E0481B590BBC01665D794FC801EC
:105C500041D5B5CD4AE150E06FEF70E0CE01079637
:105C600065D58091E5028983EA821B821C8284E0EB
:105C70008D8385E0AECD81E090E090930803809322
:105C8000070382E390E09093DA028093D9020E94A6
:105C9000420B9093D8028093D70291CDE114F10486
:105CA00081F1B090DB02A090DF02C090D702D090CB
:105CB000D8020E94420B8C199D098536910540F14E
:105CC000A5FE26C0B0FE24C00E94420B9093D802CD
:105CD0008093D7028091D9029091DA020197909334
:105CE000DA028093D902892B61F410920803109292
:105CF000070381E090E09093E6028093E502E12CB7
:105D0000F12C8091E5028983EA828091D90247CD06
:105D100082E390E09093DA028093D902F2CF10925E
:105D2000E6021092E5024BCD40E250E06FEF70E0EA
:105D3000C801FCD444CD8B81873071F0883049F1A3
:105D400081113DCD8FE1D8011D928A95E9F788E058
:105D50008C8383E088A333CD2C8166E0CE018196CD
:105D6000FC01362F11923A95E9F7283080F4629FB2
:105D7000B001112463537E4F46E050E0DED480E052
:105D8000898386E0FE01B196DE0112962FCD8FEF5A
:105D9000F7CF6C8186E0FE013596DE019196019089
:105DA0000D928A95E1F789A19AA181154CE7940794
:105DB00041F42091E5023091E602232B11F480E0BA
:105DC00090E09AA389A38BA19CA18115ACE79A07C7
:105DD00041F42091E5023091E602232B11F480E09A
:105DE00090E09CA38BA38FEF683060F4B6E06B9FCC
:105DF000B001112463537E4F46E050E0CE018196FE
:105E0000EBD480E089830E942D17D9CC2B3031054B
:105E100008F001CC2ECC8091C002811509F496CAFD
:105E2000B0E1B9BDE2E1E9BD09B400FEFDCF80916A
:105E3000D8008F7D8093D8008091E00082608093AD
:105E4000E0008091E00081FDFCCF0E94800F7ECABF
:105E50001F921FB61F9211248F939F93AF93BF93EE
:105E60008091BF02811113C0809128029091290274
:105E7000A0912A02B0912B024196A11DB11D8093E1
:105E8000280290932902A0932A02B0932B02BF917B
:105E9000AF919F918F911F901FBE1F90189578947E
:105EA0001F921FB61F9211248F939F93AF93BF939E
:105EB0008091280290912902A0912A02B0912B0290
:105EC0000196A11DB11D8093280290932902A093F1
:105ED0002A02B0932B02BF91AF919F918F911F9097
:105EE0001FBE1F9018951F920F920FB60F9211248C
:105EF0002F933F934F935F936F937F938F939F93D2
:105F0000AF93BF93EF93FF938091E10082FF09C0AD
:105F10008091E20082FF05C08091E1008B7F809339
:105F2000E1008091DA0080FF24C08091D80080FFDA
:105F300020C08091DA008E7F8093DA008091D900B2
:105F400080FFA9C080E189BD82E189BD09B400FE5E
:105F5000FDCF81E08093E70280911702811109C093
:105F60000E94420D0E94B80D8091E20084608093EF
:105F7000E2008091E10080FF1AC08091E20080FF82
:105F800016C08091E2008E7F8093E2008091E20053
:105F900080618093E2008091D80080628093D80075
:105FA00019BC85E08093E70283E08093150180911E
:105FB000E10084FF2FC08091E20084FF2BC080E1CC
:105FC00089BD82E189BD09B400FEFDCF8091D80072
:105FD0008F7D8093D8008091E1008F7E8093E100D7
:105FE0008091E2008F7E8093E2008091E2008160E8
:105FF0008093E20080911602811509F452C084E07A
:106000008093E7028091E702843009F052C082E079
:10601000809315018091E10083FF2CC08091E20004
:1060200083FF28C08091E100877F8093E10082E0B8
:106030008093E702109216028091E1008E7F809398
:10604000E1008091E2008E7F8093E2008091E20087
:1060500080618093E20042E060E080E00E94880D71
:106060008091F00088608093F00081E080931501BA
:1060700080931401FF91EF91BF91AF919F918F9108
:106080007F916F915F914F913F912F910F900FBE34
:106090000F901F90189519BC1092E70210921702EA
:1060A00068CF8091E30087FF02C083E0A9CF81E041
:1060B000A7CF81E0ADCF1F920F920FB60F921124A0
:1060C000EF92FF920F931F932F933F934F935F9302
:1060D0006F937F938F939F93AF93BF93CF93EF93E0
:1060E000FF9309EE10E0F8018081C091EC008F7001
:1060F000C795CC27C795C82B108280EFE82EF12CCE
:10610000F7018081877F808378940E94B80FF8011F
:106110001082F701808188608083CF70F801C0838E
:10612000FF91EF91CF91BF91AF919F918F917F910F
:106130006F915F914F913F912F911F910F91FF9020
:10614000EF900F900FBE0F901F9018958EE1489B17
:1061500002C08A95E1F7489BFECF0895589880E2E7
:106160008A95F1F7589A0895FC012BE02A95F1F7EA
:1061700028E090E080E031E040E14A95F1F7880FB7
:10618000489B02C08160932742E04A95F1F70000E6
:1061900040E14A95F1F72A9579F720E12A95F1F740
:1061A00029B132E03A95F1F7000040E14A95F1F764
:1061B000217092272081920F90830895A1E0B0E092
:1061C000E3EEF0E375C119828C017C01E60EF11C4F
:1061D000BDDFCE010196C8DFF80181938F01EE1576
:1061E000FF05B1F781E09981911180E02196E6E009
:1061F0007BC1509A589A08955098589AE89AE9E6BF
:10620000F0E080818C7F808308956150770B91E06E
:1062100001C0990F6A95EAF7692F90E021E06111BA
:1062200008C0911599F0589A80E28A95F1F758982C
:106230000895362F3823311539F0589A922730E2D5
:106240003A95F1F76695EBCF5898F9CF5898ECCF7F
:10625000FF920F931F93CF93DF93EC018C01060FF6
:10626000111DF9907BDF68E08F2DCFDFC017D107BC
:10627000C1F7CDB7DEB7E5E038C11F920F920FB678
:106280000F9211240F931F932F933F934F935F937C
:106290006F937F938F939F93AF93BF93EF93FF93EE
:1062A000CF93DF930F92CDB7DEB719824FDFCE01C8
:1062B00001965ADF082F069506950695982F929518
:1062C0009570202F2570920F292F23709695969503
:1062D000920F982797708981892B811509F058C0F2
:1062E000043008F055C080E18A95F1F7589A509A29
:1062F00082E08A95F1F700C0589888E0089F8001F5
:106300001124D801AD5DBE4F1696ED91FC91179703
:106310003097A9F0609190017091910114962D91A0
:106320003C911597260F371F11968D919C911297CE
:10633000680F791F13964C9113978C910995F8016A
:10634000ED5DFE4F6381611549F020919001309120
:10635000910184819581820F931F7ADFFFDE80E1B6
:106360008A95F1F758985098589A80E18A95F1F7F4
:10637000F801ED5DFE4F6081611549F020919001BB
:106380003091910181819281820F931F17DFDEDEB0
:106390000F90DF91CF91FF91EF91BF91AF919F91BE
:1063A0008F917F916F915F914F913F912F911F91AD
:1063B0000F910F900FBE0F901F9018950F931F9382
:1063C000CF93DF938C0104970CF05EC0F894509A41
:1063D000589885E08A95F1F70000C02FC695C570E2
:1063E000802F8570C80F8C2F8370C695C69593E05B
:1063F000000F111F9A95E1F7C80FC8018C2BEC0113
:10640000ADDE00C068E08C2F00DF90E19A95F1F7D7
:106410005098589A489B31C087E090E048992FC027
:10642000F801ED5DFE4F6381611559F020919001F7
:106430003091910184819581820F931FBFDE811578
:1064400001F184DE80E28A95F1F75898509A90E144
:106450009A95F1F7F801ED5DFE4F6081611549F005
:10646000209190013091910181819281820F931F3F
:10647000EFDE74DE789481E008C000C0CBCF0197D6
:1064800049F4509A589A789480E0DF91CF911F9107
:106490000F91089500C0C2CF2F923F924F925F920A
:1064A0006F927F928F929F92AF92BF92CF92DF9224
:1064B000EF92FF920F931F93CF93DF93CDB7DEB789
:1064C000CA1BDB0B0FB6F894DEBF0FBECDBF09941D
:1064D0002A88398848885F846E847D848C849B8474
:1064E000AA84B984C884DF80EE80FD800C811B8182
:1064F000AA81B981CE0FD11D0FB6F894DEBF0FBEB1
:10650000CDBFED010895992778E0880F991F961760
:1065100008F0961B881F7A95C9F780950895AA1BE5
:10652000BB1B51E107C0AA1FBB1FA617B70710F07E
:10653000A61BB70B881F991F5A95A9F780959095B0
:10654000BC01CD01089597FB072E16F4009406D0E8
:1065500077FD08D0E4DF07FC05D03EF490958195E7
:106560009F4F0895709561957F4F0895EE0FFF1F1F
:106570000590F491E02D0994082E817006940694FC
:10658000811D0694811D0694811D0694811D06942B
:10659000811D0694801D089569279627692778270D
:1065A0008727782708957DD1332312F48A1B9B0B0C
:1065B00001C077D1B7FF0895821B930B0895002E79
:1065C000083090F0982F872F762F652F542F432F68
:1065D000322F22270850F4CF220F331F441F551F9C
:1065E000661F771F881F991F0A95B2F7002D08951F
:1065F00097FD1094002E083098F00850232F342F68
:10660000452F562F672F782F892F912DF4CF159472
:1066100097958795779567955795479537952795DA
:106620000A95AAF71124002D08958F929F92AF9298
:10663000BF92CF92DF92EF92FF92CF93DF93EC0164
:10664000688179818A819B81611571058105910538
:1066500021F464E279ED8BE597E02DE133EF41E041
:1066600050E0D1D049015A019B01AC01A7EAB1E445
:10667000E6D06B017C01ACEEB4EFA5019401EBD048
:10668000DC01CB018C0D9D1DAE1DBF1DB7FF03C0EE
:106690000197A109B04888839983AA83BB839F7718
:1066A000DF91CF91FF90EF90DF90CF90BF90AF90B0
:1066B0009F908F900895B9CF80E091E0B6CFA0E091
:1066C000B0E08093000190930101A0930201B09388
:1066D00003010895FB01DC0102C005900D924150B9
:1066E0005040D8F70895FC014150504030F00190DF
:1066F0000616D1F73197CF01089588279927089575
:10670000FB01DC0104C08D910190801921F44150FE
:106710005040C8F7881B990B0895FB01DC0102C0AB
:1067200001900D9241505040D8F70895DC0101C00E
:106730006D9341505040E0F70895DC01CB01FC011E
:10674000F999FECF06C0F2BDE1BDF89A319600B4CA
:106750000D9241505040B8F70895F999FECF92BD7F
:1067600081BDF89A992780B50895A6E1B0E044E08C
:1067700050E0E5CFA8E1B0E042E050E0E0CFDC013E
:10678000A40FB51F4150504040F0CB01840F951F1E
:106790002E9105D041505040D8F70895262FF999F1
:1067A000FECF92BD81BDF89A019700B4021639F070
:1067B0001FBA20BD0FB6F894FA9AF99A0FBE089541
:1067C0000396272FECDFEADF252FE9DF242FE7CF21
:1067D0000196272FE4DFE2CFDC01CB0102C02D912F
:1067E00005D041505040D8F70895262FF999FECF93
:1067F0001FBA92BD81BD20BD0FB6F894FA9AF99ADE
:106800000FBE01960895052E97FB16F400940FD045
:1068100057FD05D024D007FC02D046F408C050959F
:106820004095309521953F4F4F4F5F4F089590957C
:106830008095709561957F4F8F4F9F4F089531D010
:10684000A59F900DB49F900DA49F800D911D1124C4
:106850000895B7FFF4CFF3DF821B930B0895A1E2F5
:106860001A2EAA1BBB1BFD010DC0AA1FBB1FEE1FCA
:10687000FF1FA217B307E407F50720F0A21BB30B15
:10688000E40BF50B661F771F881F991F1A9469F791
:1068900060957095809590959B01AC01BD01CF01ED
:1068A0000895A29FB001B39FC001A39F700D811DE9
:1068B0001124911DB29F700D811D1124911D089509
:1068C000F894FFCFAC0BB10BB30BB80BC80BC80BD4
:1068D000C80BC80BC80BC80BC80BC80BBA0BBE0B38
:1068E000C10BC60BD60BDC0BE00B9510BB10C11017
:1068F000BB10C11013113411C1103A1247126419A0
:106900005B19771959194E194E1959194E194E1903
:1069100093194E199E194E194E194E194E194E19AA
:1069200059194E194E1959194E1985194E194E19E2
:10693000B019B019B019B019B019B019B019B0190F
:10694000B01952194E19641958195E20C6206620D4
:10695000302034206A2038206E207A204420BF2046
:1069600048207E204C208220A72050208620AE2068
:1069700056208C2094203C207220402076205A20E3
:1069800090209E20B720BD202A206220CD20072005
:106990000B20FE1F03200F2013201720EE200721BD
:1069A0000C21112116211B21202125212A212F21F3
:1069B00034219E229E22D822D8228C23A723002372
:1069C0000023AC23212434243424DA2DF12DF82D96
:1069D000DF2BDF2B2A2E3B2E4E2E8F2E942EDF2BDD
:1069E000DF2BDF2B9B2ECD2BD12BFB2B072C122C3F
:1069F0001D2C202C592C7B2CCA2BC62D822C852C8F
:0C6A0000892CB42CF02CF32CF52C2A2D42
:106A0C000100000001010201191A1B1C1D1E1F2090
:106A1C00212200000100013F0B990E980CAF0EB41F
:106A2C000E900E00000001000000000000000501A7
:106A3C00000000040600000000000028081E0A14D4
:106A4C00014663C879DA3393C20044227B4901279B
:106A5C0001AC004F02680288020001020202020629
:106A6C0006060909090909090F0F0F0F0F0F151554
:106A7C001518191919191919191919192324252552
:106A8C00252525256697C63435323331F7F69436ED
:106A9C00EC02E200E900EA00B500B600B700CD0058
:106AAC008301CC008A019201940121022302240269
:106ABC002502260227022A02B300B4006F007000E0
:106ACC009F01CB019F02A002E200E900EA00B500A1
:106ADC00B600B700CD008301CC008A01920194016D
:106AEC002102230224022502260227022A02B300D5
:0E6AFC00B4006F0070009F01CB019F02A0024A
:00000001FF
